:020000041100E9
:10300000002370B5284C0120636101F03FFA402095
:103010000223FE21254A207401F0BEFA002833D194
:103020000223FF21224A207C01F0B6FA00282BD18E
:10303000204BA2899A4224D1E3891F4A93420CD1A2
:103040001E4B63611E4B2268002A03D1002B01D066
:1030500023CB23C401F08EFA70BD1A4A934201D0EB
:103060000023F0E7184B194A1B68934205D9C02288
:103070000421207C920001F009FB104B6361144B8A
:10308000E1E700232374EBE7CC223820AC21920146
:10309000207401F0FBFA0028F3D10E4B63610E4B54
:1030A000E3810E4BCFE7C0469863FF1FA463FF1F69
:1030B000A663FF1F5959000083050000ED4200116F
:1030C00034BE001182150000BC63FF1F871300008F
:1030D00040BE001189430011AAAAFFFF28BE0011BB
:1030E000F7B5164B0192C318021D002000938823E8
:1030F0005B05D3181B685C1C1AD09CB2402C18D8F6
:103100008D781E0CAC466746CD782D023D43AE420D
:1031100006D1019800280ED110000C70240A4C70C2
:1031200003249BB20733A343D218009B9A42DED3F9
:10313000FEBD4432F9E71000FAE7C046FC0F00007C
:10314000802213B503000324019189B25201073193
:103150009B18A14304305A1A88235B05C3181B68C7
:10316000591C03D190429241104016BD99B240299A
:1031700007D80B000733A343C0189042ECD30020BC
:10318000F3E74430F9E7134B134A1B68126810B594
:10319000FA24934201D81A00F824104BE4021B6869
:1031A0009A4210D813000E4A12689A420ED3013385
:1031B00007D1F823DB029C4203D10A49054808F0F5
:1031C000D7FC200010BDFC24E402ECE7FE24E4025E
:1031D000F7E7C04600C0071100D0071100E0071153
:1031E00000F00711FFFFFF7FF0B59BB015000490C2
:1031F0000391402A00D9A0E006AB59801A80FFF75E
:10320000C2FF0400042816D9002206A9FFF768FFB0
:10321000052810D906AB1B88AB420CD1002D07D076
:10322000514B2A000499C01808F01AFD002802D159
:1032300001201BB0F0BD06AB1D8020000699FFF7F2
:103240007FFF041E7BD1069B0793FFF79CFF802323
:103250005B01C618802307001B039E4201D3F8269A
:10326000F60288235B05F31801931B68013302D033
:10327000019808F0F5FA3D49019808F079FC3B1DEA
:103280000293331D05938822029B52059B181B68ED
:1032900008935A1C3CD044219AB20091402A04D889
:1032A0000320D11D814389B2009103991B0C8B42ED
:1032B00024D0402A22D80122300008A9FFF710FFAD
:1032C000021E1BD1380008A9FFF70AFF04000428DA
:1032D00031D9009A059B9B1880225201B218934263
:1032E00040D288235B05C118009A09A808F0F0FBBA
:1032F0001D4B009A09A9F01808F0DAFA009A029B0F
:103300009446634402931A4B029AFB189A42BAD32A
:1033100088235B05FC1821680198013908F028FC16
:10332000200008F09DFA039A07AB5A8030000799F5
:10333000FFF706FF0400002C03D1002079E70428E2
:10334000FBD988235B05E018069908F011FC0323DC
:10335000EA1C9A4300D16BE7034B0499E01808F08C
:10336000A7FA65E70424ECE704000011FFFFFF7FE4
:10337000F80F0000F7B505001400402A21D80027F7
:1033800001AE71803780FFF7FEFE042816D93A009F
:103390003100FFF7A5FE042810D93688BC420BD0B7
:1033A000BD4209D0221CB44200D9321C064B92B255
:1033B000C118280008F08CFB30B2FEBDC04300B23B
:1033C000FBE703204042F8E70400001137B5042270
:1033D00004000D0001A81649FFF7CCFF02000428E5
:1033E0000BD1019BA34208D3AB4204D0104901A8E2
:1033F0000195FFF7F9FE01203EBD0E4C2368200029
:10340000019308F02DFA019920000139019108F08B
:10341000AFFB80235B01E418074B9C42EED10422F2
:10342000034901A80195FFF7DFFE0020E4E7C0464D
:103430005555000000C007110000081130B589B0D3
:1034400008F0EEF910226946254808F091F9254B5D
:10345000009A9A420ED1019B029A0F2B33D8002179
:1034600001240698013B08D2002900D00292029B59
:10347000013331D10023029325E0551CF2D1020023
:103480002100EFE710341022200004A908F070F9A1
:10349000029B013301D1069B0293882304995B05AB
:1034A000C918059B06981A03120B049105928142D4
:1034B00003D02B4201D108F00BFB019B013B019390
:1034C000019B002BDED1029B002B03D004930498B8
:1034D0004168084709B030BDE025014C2D03EFE7F6
:1034E0000000011150485936F7B50F490F4B0A68D3
:1034F00004001A4084235B0013430B60030003277E
:103500001033019300252E00112008F0C1FA084B5A
:103510001B683B40AB4002351E43202DF4D1019B7C
:1035200040C4A342EED1F7BD5CF0004000FEFEFFB8
:1035300064F00040802270B5AD4CAE4BD20000214B
:1035400020001C6008F064FB2300AB4A88331A603B
:10355000AA4B1A786E23002A00D01133E3620A23A3
:103560002365A74B1878A74BA0630138E361C3B26A
:10357000032B01D810232362A34B37226361C82396
:10358000DB00A36123008C331A60082336210F3A35
:10359000E518E16323646264E9670439251DE9677E
:1035A00025003B26BC352E602500C0352B6025004C
:1035B000C4352A6025000636CC352E602500083E2D
:1035C000C8352E602500D03529602100D4310B602C
:1035D0002100D8310A6021000225E0310D6025006C
:1035E0004221DC35296025001B3EE4352E60250094
:1035F000E8352B602500EC352A6022000525F432E1
:1036000015602200F03211602200183190321160F2
:1036100022009432136023003C2298331A60AF23B7
:10362000DB002360794B2363032805D808F080FA78
:10363000330235371523636096232100FA225B009D
:10364000A360E360C8332361714BFC319200A36433
:103650000A6062626F4A704DA2627322E2656D3A3F
:103660006265A2650232E5644A60022161669621C4
:103670008900A166626709210022E166A2676749A5
:10368000674A684E2167E2673560032811D808F061
:103690004FFA96089EA61023CDE70E23CBE70C2306
:1036A000C9E720001A259C30056020000735A030AE
:1036B00005602000A83003602300FA20F833800062
:1036C000186023006420A433186023005F38AC33F3
:1036D000186023000338B03318602300C630B433B9
:1036E000186023000020B833186023003825FC330D
:1036F0009D604D4D5A665D644C4D9A64DD61962522
:10370000AD001D624A4D9A675D62F53DFF3D9D62C9
:103710001E25484ADD6618675867D9651966DA6755
:10372000BE23C021444A5B00E250444B4900635031
:1037300004316250C4225200A350FA23E4205B00FB
:103740000432A3500432A3503D493E4A3E4BD1605F
:103750003E49800019503E49E938FF3819503D492B
:10376000043019503C491038D1613C4911633C493F
:1037700051633C4911603C49195019003B48F831EC
:1037800008603B49D16582213A4A89005A501A00A3
:1037900039490832D1671A003849B432116088219A
:1037A000374A89005A501A00364988321160364A21
:1037B000DA6408F0D5F8012008F0AAFA70BD2000FC
:1037C00014259C30056020000435A03070E72000EF
:1037D00010259C30056020000335A03068E72000EC
:1037E0000E259C30056020000235A03060E7C04601
:1037F0000004FF1F7466FF1F6071FF1F2C46FF1F30
:103800004A0AFF1F3A07000080C3C9019A0200005C
:1038100050C300006A180000280A0000204E000073
:1038200088130000F009FF1F00400011681000001D
:10383000C4090000DC05000040420F001027000012
:10384000FD1BFF1FFC00FF1F0000FF1F2D2FFF1F90
:103850005532FF1FED30FF1FE11FFF1FFD1FFF1F30
:10386000A921FF1F491FFF1FCD28FF1F952CFF1FF8
:10387000D918FF1FD927FF1F4125FF1F4D25FF1F07
:10388000491EFF1F011FFF1FC11DFF1FF7B50B0CB6
:10389000FF270122009300233C001E001D009446D8
:1038A000019089B262469A401000084018413618CB
:1038B000B6B2FF2F02D1012E00D19FB20098024074
:1038C0001A41AD18ADB2FF2C02D1012D00D19CB22E
:1038D0000133102BE6D10320012E07D1012D04D195
:1038E000019B2401E4191C700138FEBD102EFCD18F
:1038F0000238102DF9D00230F7E710B5064C2378C6
:10390000002B07D10548FFF7EFFD0548FFF7ECFD59
:103910000123237010BDC0463466FF1F4866FF1F99
:103920003866FF1FF0B58BB00D0001230190102900
:1039300036D8FFF7E2FF00231A001B48C15C0133B1
:103940005218102BFAD1023B002A29D0174B184CE1
:103950001F68002306A9E25C1600FA5C56405E541C
:103960000133102BF7D102AA07F0B2FE2A0002A9F8
:10397000019808F05DF908F00BF923681B18236023
:1039800008F006F963681B18636008F001F9A36882
:103990001B18A36008F0FCF8E3681B18E360002321
:1039A00018000BB0F0BDC0464866FF1FCC44FF1F97
:1039B0003866FF1F0223F0B501245D4D5D4E2B706C
:1039C0005D4B91B01C705D4F039333680820BB7052
:1039D00006F03AFC0023984205D0BA78552A02D066
:1039E000332A00D098E03360002006F0ADFE08F0E6
:1039F00097F9FFF79FFD08F07BF81F2201240021B3
:103A00004F4B10AE1A704F4B1C704F4B19704F4BF1
:103A100019689143163A0A431A6060221968914363
:103A2000403A0A431A6007F07BFF07F0E1FFC1202C
:103A3000FF21474B80001A588A431A50C522920032
:103A400098588843BF3901439950985841490840D4
:103A50008021C9010143802099509958C00509026D
:103A6000090A0143995080213B48490107F0A8FF0A
:103A700003232200394901940093394808F010F8D3
:103A80002C22384905A808F023F805AC6178207885
:103A9000023406F0F9FBA642F8D10121002006F01D
:103AA00007FD314B314A196803201140A022D20290
:103AB0000A431A608022196892040A431A6019683E
:103AC0002B4A1140802292030A431A60294B2A4A4A
:103AD000934200D8012007F09BFF08F009F907F096
:103AE00037FF287807F054FF039B1878C0B208F01E
:103AF000AFF807F0CDFD2149042007F0E9FE06F0FC
:103B0000EFFD00F0AFF800F01BFE00F0ADFE00F09E
:103B100019FA002011B0F0BD00932100174A0420CB
:103B200008F0AEF88023DB059C62FFF787FC5BE7BB
:103B30004A0AFF1F34F000402C46FF1FC863FF1FD6
:103B4000480AFF1F490AFF1F680AFF1FBCF0004018
:103B500000E100E0FF00FFFF3046FF1FB458FF1FE9
:103B60003056FF1F50BD001114F00040FF7FF8FFDA
:103B7000FFFF9FFF6071FF1F0080FF1F3B000108D8
:103B800070B500252849294A29484D6308CA1B05F4
:103B90001B0DED188242F9D10022264B8B63264B78
:103BA00008211A628022254B9205DA67244BDA68D5
:103BB0008A43DA60234A1278012A03D09A6822499C
:103BC0000A409A600121EE242048E40002686C4318
:103BD0008A430260DA6811208A43DA6008F020F82C
:103BE000112007F015FE112007F02AFF184A200CBB
:103BF0000400642390420AD8FA220023D2009042A3
:103C000005D9144B0A21C01807F02AFFC3B2124A83
:103C10001372124BD4801B78002B04D1104B10214F
:103C2000187807F04DFF70BD00000540880505407D
:103C300000060540FF01000000F0004004E100E044
:103C40003CF000404A0AFF1FFFDFFFFF0038004042
:103C5000B70B000030F8FFFFB063FF1FEC65FF1FDC
:103C6000E863FF1F002210B51100112007F0A8FF24
:103C700010BD0000F8B5002301250826394F3A4C45
:103C80003B62E3681120AB43E360E368B343E36066
:103C900007F0BEFD112007F0C3FF112007F0F8FD6B
:103CA0004023226829001343236080236268DB02DB
:103CB000134380226360A36807201343A360A368B3
:103CC0002A4A1340A3608023A2689B011343102259
:103CD000A360236C93432364236C2B4323648023CE
:103CE0005B003B62226B224B1A402263626B1A40DC
:103CF0006263A26B1A40A263E26B1340E3631D4A46
:103D0000E3681340E36006F0A5FB2900072006F0F6
:103D1000CFFB8021184A1120536C0B43536407F0EA
:103D2000DFFEFD21154B164A89005A508023C7201B
:103D3000626B5B0313436363E36880003343E360B8
:103D4000E368104A1D43104BE5601958114080226A
:103D500012020A431A50802292051A600B4B5E63CE
:103D6000F8BDC04600F000403CF00040FFFFDFFF20
:103D7000EFFFEFFFFFFF7FFF003800400000FF1F55
:103D8000813B0011FF00FFFF00E100E00000054063
:103D900030B503A804880B20002C0ED14968074DCC
:103DA00008784978090201430A20A94205D1012176
:103DB00020001980024B1B7A137030BD192A0000B5
:103DC000B063FF1FF7B5150008AA16884A680F4FA1
:103DD00014785278120222430A24BA4214D10122E2
:103DE000DBB2019200962A0007F0CAFB041E0BD139
:103DF000074B1B68002B07D068782A780002104315
:103E000042425041013098472000FEBD0229000087
:103E10003463FF1F30B5012503790400BFB02B4286
:103E200012D00A49408806F017FF28420CD06A4693
:103E3000074B69465B8D55801380064B60881B7A63
:103E40001371002203F0E8FF3FB030BD2C63FF1F69
:103E50007042FF1FB063FF1F10B50549054806F00B
:103E6000B1FE0421044A054806F06EFE10BDC046AE
:103E70002C63FF1FFFFF00007CBD00117042FF1F7D
:103E800010B5024804F04AFE10BDC046153E0011B0
:103E9000062310B5837010330371443B43712A33FA
:103EA00083714433C37100230222012103720E4B3C
:103EB000027041701C8881724472197A0273C17257
:103EC0009A784273DA7882730322C2731A79027481
:103ED0005A7942740C2282749A79C274DB79037520
:103EE0001123C370152010BDB063FF1F10B514203F
:103EF00007F07EFC124B14220021186007F088FEA8
:103F0000002007F06DFE012007F07AFC022007F088
:103F100037FE032004F0A6F8042006F0BBF80520C5
:103F200003F0E4FA062003F0B1FF072001F0C4F922
:103F3000082006F0E9FD092000F09EFF10BDC046F4
:103F40003863FF1F10B507F0ABFB012007F030FD11
:103F500007F0C6FE002010BD094B10B504009842C2
:103F600005D0012904D12000064906F02BFE10BD22
:103F70000229FCD1013904F08FFD0028F3D0F6E7C7
:103F8000FEFF00005E63FF1F70B50D7A100004AAEB
:103F90002C00168810221440154220D1002E20D16A
:103FA0000A78022A18D14A68517815780E4A09020F
:103FB0002943914205D00D4A914209D01C800A2420
:103FC00004E014220A491A8007F082FD200070BD27
:103FD0000C2208491A80F7E71C800124F6E7082420
:103FE000F4E70B24F2E7C046F3FF0000F4FF000003
:103FF000B044FF1F58BE001110B50400074908481F
:1040000006F0E0FD074804F0C9FC0020E40704D5F1
:104010000721054A054806F097FD10BD5E63FF1FA6
:10402000FFFF0000593F0011C0BD0011B442FF1F47
:1040300000B50C4BBFB01A780B4901A800F046FC44
:104040006B4680B25880002809D06A46074B694603
:104050001B881380064B0022188803F0DDFE3FB05A
:1040600000BDC0463C63FF1F3D63FF1F0E43FF1FA3
:104070000E44FF1F00B50C4BBFB01A780B4901A8C6
:1040800001F010FE6B4680B25880002809D06A46C5
:10409000074B69465B8D1380064B0022188803F09E
:1040A000BBFE3FB000BDC0466663FF1F6763FF1FD6
:1040B000B442FF1F0E44FF1FF7B50E00377A1C00F5
:1040C00008AB11003D001A8820231D401F423CD13F
:1040D0003378022B3BD173681F785B781B023B431C
:1040E0001E4FBB4208D01E4FBB4214D01D4DAB42E9
:1040F00021D00A252800FEBD002A2AD1142C2AD856
:104100002200F06807F0E4FC174B1C70012CF1D979
:10411000FFF7B0FFEEE7002A1BD1202C1BD82200AE
:10412000F06807F0D5FC114B04211C70104B187877
:1041300007F0C6FCDEE7E3B20124009201940A0016
:10414000310007F01DFA0500D4E70825D2E7012564
:10415000D0E70B25CEE70D25CCE7C046F3FF0000E6
:10416000F4FF0000022900006663FF1F3C63FF1F8D
:10417000E863FF1F332310B5040003700A220749C8
:10418000013007F0A5FC064B0F201B681A0AE372EA
:1041900022731A0C1B0E6273A37310BDB063FF1F52
:1041A000D863FF1F30B5012503790400BFB02B424F
:1041B00013D00B49408806F04FFD28420DD06A46C7
:1041C000084B01A81B881380FFF7D4FF6B4658806B
:1041D00000226946608803F01FFE3FB030BDC04634
:1041E0005E63FF1F0E43FF1F10B5024804F096FCEC
:1041F00010BDC046A541001170B5160004AA148870
:1042000005AA15784A685078117800022A4A0843AE
:10421000801805284BD807F08BFC03131E29343F68
:104220000720032C0BD80422121BAA4200D92A0013
:1042300022491A803000091907F04AFC002070BD9D
:104240000720112CFBD81222121BAA4200D92A00E7
:104250001B491A80EEE707200E2CF0D80F22121B04
:10426000AA4200D92A0017491A80E3E70720032C45
:10427000E5D80422121BAA4200D92A0012491A804A
:10428000D8E70720032CDAD80422121BAA4200D94F
:104290002A000E491A80CDE70720032CCFD804222C
:1042A000121BAA4200D92A0009491A80C2E700223B
:1042B0000A201A80C3E7C046DCD5FFFF0BBE001101
:1042C0008463FF1FFBBD0011F6BD0011F1BD00119D
:1042D000ECBD001110B50D21024A034806F034FC74
:1042E00010BDC046E0BD00112443FF1F37B50020BC
:1042F00000F0CCF8204D214BEA89287C9A422AD143
:10430000042201A900F076F9040000F033F9002C32
:1043100030D16B4699882B68C9BA4B432989184A12
:104320001B145B1853806B46D9886B6849BA89B2F5
:104330004B4369891B0C5B181248191C1BB2834242
:1043400000DD011C0B0400D500211388918001338E
:10435000138020003EBD0223002101AA00F01CF9B9
:104360006A46040002230121287C063200F014F979
:104370000443CAE70124ECE79863FF1F83050000AC
:10438000B063FF1F0F27000037B5012000F07EF853
:104390001F4D07226946287C00F02CF9041E33D1FA
:1043A0006B461B787F2B2FD800F0E4F86B46D8784B
:1043B000F02302041B031A406B469B8815495BBA25
:1043C0009BB21A432B68000953432A891B0C9B1884
:1043D0004B806B465A789B7812031B011A436B681B
:1043E000024353436A891B0C9B180B481A1C1BB2CF
:1043F000834200DD021C130400D500220B888A8052
:1044000001330B8020003EBD00F0B4F80124F9E731
:104410009863FF1FB063FF1F0F27000010B50F4CFC
:10442000237C002B0CD0382B0BD1012000F02EF870
:10443000CC22AC21207C920100F028F900F09AF8FF
:1044400010BD074BE2899A42FAD1012000F01EF814
:104450000021207C00F0FAF8F0E7C0469863FF1FC7
:104460008305000010B5084B1A7C002A09D05B694F
:10447000002B06D09847041E01D0FEF7C1FD200096
:1044800010BD0124F9E7C0469863FF1F70B50021F5
:104490000600162006F042F80121152006F03EF82D
:1044A00007F036FB0400092007F0F2F900222B4B3D
:1044B0002B4DDA6661321A6019685B3A9143002E1F
:1044C00028D0023A0A431A60AC4209D10A22DA61C2
:1044D00007321A6200221A639A630132DA6370BDEE
:1044E000204A944203D11E22DA610532F1E71E4AC6
:1044F000944203D13022DA610632EAE71B4A944241
:1045000003D14322DA610832E3E7194A9442E1D148
:104510006922F7E702220A431A604622AC4203D01E
:10452000104A944204D194225A6106329A61D1E72A
:104530000D4A944201D1E622F6E70C4A944204D196
:104540003422FF325A610D32F0E7094A9442C1D158
:10455000E62252005A610A32E8E7C04600500040A5
:104560000024F4000048E801006CDC020090D00355
:1045700000D8B80510B50024064B0920DC6607F00A
:1045800047F92100162005F065FF2100152005F0F0
:1045900061FF10BD00500040F8B51C000023134D12
:1045A0000F00EB666860160007F03AF901238022DD
:1045B000EB6623002F615200013B08D207F058FB45
:1045C00008200B4A1168002C03D12000F8BD2A6195
:1045D000F2E72B6F034203D02B69013C33700136A5
:1045E00013685B1A032BEED90124EEE7005000405C
:1045F0006008FF1F002370B5124D1400EB66686061
:104600000E0007F00DF901238022EB662300520013
:10461000013B08D207F02CFB08200B4A1168002C44
:1046200003D1200070BD2A61F2E72B6F034203D053
:104630002B69013C3370013613685B1A032BEED9EA
:104640000124EEE7005000406008FF1F002370B512
:104650000C4C0D00E366606007F0E2F80123E366AE
:10466000256107F005FB8020074A80001168636B15
:10467000034205D113685B1A032BF8D9012070BDE2
:104680000020FCE7005000406008FF1F002370B5C9
:10469000134C0E00E3666060150007F0C1F80123BB
:1046A000E36626610F33626B1A42FCD02B0A23614A
:1046B0001023626B1A42FCD0EDB2256107F0D8FAE4
:1046C0008020084A80001168636B034205D113689B
:1046D0005B1A032BF8D9012070BD0020FCE7C0460F
:1046E000005000406008FF1F002370B5124D0C0001
:1046F000EB666860160007F093F80123A619EB66D5
:104700000F33B4420ED107F0B3FA80200B4A800079
:1047100011686B6B03420CD113685B1A032BF8D939
:10472000012070BD22782A616A6B1A42FCD00134E4
:10473000E7E70020F5E7C046005000406008FF1F93
:1047400010B5084CE368002B08D1074B1B685B04CD
:104750005B0C0A336360054B1B68236006F0D0FFD7
:10476000A06010BDD863FF1FC8F00040CCF000402F
:1047700010B507F055F80F4B996A9A6A8A42FBD137
:104780000D4C6268A0688A18121A531E884200D322
:104790001300A1602168DA0B52185B0407495B0C17
:1047A000636022600B60064B1A6007F061FA2068B4
:1047B00010BDC04600F00040D863FF1FC8F00040A5
:1047C000CCF0004070B51F4C23793F2B01D93F231B
:1047D00023711D4B22791A701878C0B207F080F847
:1047E00018231A491A4A0B801A4913800B805380E8
:1047F000A379194980200B800C21938001334B430E
:104800000001191C834200D9011C144BD18019806E
:104810006379002B11D101336371237A012B01D805
:10482000022323726279237A0D4853430A215843A5
:1048300007F016F90B4D286070BDA02BEDD9A02311
:10484000EAE7C046CC63FF1F480AFF1F0C44FF1F66
:10485000D845FF1F0A44FF1FB865FF1F0844FF1F0C
:1048600071020000BC63FF1FF8B512210020FEF7A3
:10487000ADFD114C011E114D09D10C22104BC1CBC5
:10488000C1C4280007F0C4F9FFF79CFFF8BD0C2253
:1048900020000C49FEF76EFD0C2802D0084B43CBDC
:1048A00043C40C2228000849FEF764FD0C28EBD015
:1048B0000C220021E5E7C046CC63FF1F9863FF1F71
:1048C0004CBE0011FC0C0000F50C0000F0B50025FA
:1048D00004000E0085B0AA4268D04B1C08780193F2
:1048E0004B788978377909021943F3783F061B041E
:1048F0000B431F43039720706570262800D190E07A
:104900001CD8102812D806F0BBFF4B00FE00310067
:10491000310031009600A4009D00310031003100CB
:1049200031003100310031003100E400232800D192
:10493000BEE025285DD0FF23637099E0602800D198
:10494000A1E00AD8552834D056284CD03328F2D1CB
:104950002000FFF70FFC050028E0722800D189E055
:10496000DC2800D1EEE0712800D179E0DB2800D00E
:1049700003E1042ADFD91025052A05D0551F2A0096
:104980003800711D07F0A4F805223100200007F05F
:104990009FF82A003900601D07F09AF8053505E0F8
:1049A0000C222000854907F093F80C25280005B05B
:1049B000F0BD013A824D0C2A13D8002A0AD02800F3
:1049C000019907F085F8FFF7FDFE0C2228007D49CC
:1049D000FEF70AFC29000C22601C07F079F80D256F
:1049E000E4E70C22EBE7764D774B2A0043CB43C23A
:1049F000E9E7013A754D0C2A11D8002A08D001992F
:104A0000280007F065F80C2228007149FEF7ECFB3E
:104A100029001322601C07F05BF81425C6E70C225E
:104A2000EDE76A4B2900132218001D0007F0F0F88B
:104A3000FEF7E6FAECE705226649601C07F048F845
:104A40000625B3E712226449601C07F041F81325DC
:104A5000ACE708226149601C07F03AF80925A5E790
:104A60007178F72900D966E75D4B188801F076FD6B
:104A700002259BE75B4B012A03D072785A70627063
:104A8000F6E75B7858E7013A574D062A0ED8002A18
:104A900005D00199280007F01BF801F02DF8290036
:104AA0000622601C07F014F807257FE70622F0E7CE
:104AB000042A04D94D4D2F6006F022FEA860FFF7AE
:104AC00057FE0422039003A9601C07F001F8052596
:104AD0006CE7474D062AE2D906222800019907F023
:104AE000BFF80028DBD006220199280006F0F0FF6D
:104AF000062240492800FEF777FB0123394A517806
:104B00000B435370CBE7931E3B4F1A2B04D873789B
:104B1000002B09D100F024F9384B39001D78601CB6
:104B20006A1E06F0D5FF41E7551E2A00019938009C
:104B300006F0CEFF3249AAB23800FEF755FB00F06E
:104B400045F9E9E7022A00D8F5E67378BFB2637049
:104B5000B378A370032A05D0033A390092B2F01C4F
:104B6000FEF742FB10223900E01CFEF703FCC51CD7
:104B7000002800DB1AE760707AE7DA2800D0DAE66E
:104B8000042A00D8D7E6082A15D9B37972791B020E
:104B90001343F27912041A43337A1B0613433B6022
:104BA0003B68052231002000039306F091FF0422A8
:104BB000601D03A950E7FE236370F1E758BE0011A2
:104BC000CC63FF1FFC0C00004CBE00119863FF1F5C
:104BD000F50C0000A463FF1F8463FF1F4C45FF1FFB
:104BE0000E44FF1FC863FF1FA944FF1FD863FF1FA8
:104BF0006509FF1FADAC0000CB65FF1FC965FF1F36
:104C0000AEDE000070477047020010B5094B0A3253
:104C1000094C92B2DA815A8298811882207802F087
:104C200003FB0422054B012120781A7006F048FF8F
:104C300010BDC046D644FF1F1666FF1F1566FF1F36
:104C4000013870B5042809D806F072FF0309280856
:104C50001200234B0221187806F032FF70BD204B62
:104C60000821187806F0CCFE00221E4B1A72F5E7D8
:104C7000802200241B4B1A4D52001A8108211A6809
:104C80002878DC7207F00CF82100287806F040FD47
:104C9000012000F069FE00F02FFFDFE7104B082134
:104CA000187806F0ADFE1048FFF7F2F80F4B104AE7
:104CB0009B79002093800F4A13808022094B520079
:104CC000D8721A8100F050FE00F016FF0A4B5B7894
:104CD000002BC3D0094A136006F082FEBEE7C0462F
:104CE000E863FF1FBC63FF1F1744FF1FCC63FF1F58
:104CF000D845FF1FB865FF1FC863FF1F34F0004091
:104D000010B501290BD1082809D1054B1B78002BC0
:104D100005D02622034B04485A72FFF775FF10BDD9
:104D2000EC65FF1FBC63FF1FC40900000300F0B562
:104D30000A4D8E18B14202D152008018F0BD0C7895
:104D40002F6824093C5D0F271C700C7801313C4012
:104D50002F683C5D5C700233ECE7C0460444FF1FE3
:104D60000D22114B10B51A700C23104C10492370F2
:104D7000093A033B0F48637006F0AAFE2D23012277
:104D80000D490E48A371FFF7D1FF01220C49FFF72F
:104D9000CDFF01220B49FFF7C9FF00220A4910008D
:104DA000FEF722FA10BDC046E865FF1FC965FF1F68
:104DB0000BBE0011CB65FF1F6709FF1FD065FF1FEA
:104DC0006609FF1F6509FF1FAEDE000070B5124CBB
:104DD000132220001149FEF7CDFA114D002817DDEE
:104DE000AB78002B14D0431C2B7009236B7000236D
:104DF00000190370287829000130C0B206F0F8FECF
:104E0000297822000139C9B2002005F0BBFD70BD30
:104E1000FFF7A6FFEEE7C046CB65FF1FAEDE000042
:104E2000C965FF1F10B5114B1A781870002A0ED0F3
:104E300000280BD10E4B1A78062A07D85423D340EA
:104E4000DB0703D50B4B187802F0EEF910BD0028F4
:104E5000FCD0074B1B78012B02D0033B022BF5D86B
:104E6000044B0121187806F02BFEEFE7EC65FF1FDD
:104E70001566FF1F1666FF1F70B5514E514A524905
:104E80003070082005F00AFC0121022005F010FB1B
:104E9000022005F0F1FB0121002005F009FB0020B4
:104EA00005F0EAFB00F0A2FEFEF7AAF806F048FEC5
:104EB000032246494648FFF739FF2D240300042208
:104EC0001C7044490130FFF731FF30230470424D1C
:104ED000424C437083702E3B062220004049EB87F2
:104EE000FEF748FA062813D0200006F0C1FD02287C
:104EF00009D00321200006F0A3FE8D23E3706E3B52
:104F0000237119336371062220003549FEF76CF9CD
:104F1000344B1B68FC335C64FFF758FF0020FFF73D
:104F200081FF314C314A0121314B1278207802F057
:104F30003DF9304A304B12780021207802F036F9E2
:104F400001222E4B1A702E4B9B78552B31D12D4BB5
:104F50003B325A722C4B2D4AAB81EA812B826A82FA
:104F60002021307806F0CCFC0120404205F056FDAF
:104F70000120404205F0F2FDFFF7ACF9FEF76CFFAF
:104F800000F0A6FC01204042FFF736F8012006F0B1
:104F900097FCF72001F0C6FA0121307806F090FD69
:104FA000307802F09DFA1A4806F0BAFDFEF762FE6C
:104FB00070BD6422174B5B7953431A000A32CBE76A
:104FC000E863FF1F054C0011014D00114C45FF1F08
:104FD0008463FF1FA463FF1FD644FF1F6509FF1FE3
:104FE000ADAC00007466FF1F1666FF1F3644FF1F3E
:104FF0001744FF1FE865FF1FC965FF1FBA65FF1F44
:10500000C863FF1FBC63FF1FC4090000CE09000076
:10501000EA63FF1FCC63FF1FF8B50A0020230D00D1
:105020001A40194257D0574B1B78002B50D0FFF72E
:105030009FFB554B554C564E99686268737A8A1A95
:10504000DB039A4202D36160FEF714FE327A217AC2
:10505000531EDBB2994205D1FFF7E0F9002000F0C2
:10506000BFFD0FE09142F9D300232372FFF7FAF955
:10507000012000F0B5FD474F3800FEF709FF390069
:1050800006F046FC637A002B1FD0013BDBB2637253
:10509000002B1AD1404B9B78552B01D106F0A0FC78
:1050A000E37A002B0CD000233C4A3A4FE37213887A
:1050B000380001331380FEF7EBFE390006F028FCC0
:1050C000642370795843FFF79FFD237A01332372DD
:1050D00020206840F8BD0BB2002B0ADA304B18785C
:1050E00006F05EFD002801D006F032FB80200002B1
:1050F000EFE70224214206D0244B01201A72FFF769
:1051000091FE2000E5E70B071ED5FFF731FB1E4B94
:105110001E491F4C98684A68637A821ADB039A42D8
:1051200002D34860FEF7A6FDFFF79CF9FFF776F97A
:10513000012000F055FD00F0E5FB2368DB0701D5F9
:10514000FFF752F80820C4E71024214206D00D4B87
:105150001B78002BD5D1FEF793FED2E70124214224
:1051600007D0104800F06CF806F062FB00F0ECFC91
:10517000C7E70424080020402142ABD0FEF758FFC7
:10518000BFE7C046EC65FF1FD863FF1FBC63FF1F6E
:10519000CC63FF1F1744FF1FC863FF1FB063FF1FCF
:1051A000E863FF1FFC43FF1FF0B51B4B1B4F1B8821
:1051B0003A8804001A4E1B4D85B09A420DD83288A9
:1051C0009A420AD3184B1A882B889A4205D1174A5B
:1051D000174B12881B889A421BD0052001F0F8F962
:1051E0003B8802AA13803388019053802B88114D8D
:1051F00093800F4B02A91B88D3800F4B2A78188805
:1052000002F014FF0D4B08212878019A1C7006F05B
:10521000BFFA05B0F0BDC046B665FF1F0C44FF1FC6
:105220000A44FF1FB865FF1FB465FF1FB265FF1F6B
:105230000844FF1F1666FF1F0E44FF1FB065FF1FC7
:1052400013B50C4B1C78002C11D1002801D00A4B4F
:1052500018600A4A0A4B11780A4A10780A4A0192E1
:105260000A4A0092002205F085FA200016BD11249A
:10527000FBE7C0461566FF1FAC65FF1F1466FF1FE6
:105280000466FF1F1666FF1FF065FF1FF465FF1F12
:1052900010B5064B12201B78052B06D1044B1322A8
:1052A0001988044B187801F06FFB10BD1566FF1FBD
:1052B0000E44FF1F1666FF1F10B500240122114B7C
:1052C00052421870104B1C70104B1A8002F008F9F3
:1052D00004220F4B21001A700E480C3206F090FC8D
:1052E000102221000C4806F08BFC07220B4B1C609F
:1052F0000B4B1C700B4B1C700B4B1A700B4B1C7028
:1053000010BDC0461666FF1F1566FF1F0E44FF1F27
:105310001466FF1F0466FF1FF465FF1FF065FF1F83
:10532000C865FF1FC765FF1F1044FF1FC665FF1F2D
:10533000F8B5174C0600257806A814240078052D2A
:1053400023D1B41F134FA5B21824BD421DD88D1F01
:10535000ADB2BD4219D8FA256D00AA4215D21D0082
:105360000D4F0A3DADB2BD420FD80C4C26800C4CFF
:1053700021800C4900240A800B4A1380FFF714FF98
:105380000A4B0421187806F03BFB2000F8BDC0460C
:105390001566FF1F790C0000750C00000C44FF1F00
:1053A0000A44FF1FB865FF1F0844FF1F1666FF1F52
:1053B000F0B50BB20D0089B0002B00DB70E1A44EFC
:1053C000307806F0EDFB041E50D00378A22B00D1FC
:1053D00022E1D02B1AD0912B45D143780E2B42D10C
:1053E0009C4B82889A423ED19B4A83681278052A58
:1053F00039D1032018567F2835D0984B1B68002BD5
:1054000031D05B68002B2ED098472CE0807807289D
:1054100029D806F08DFB0428183F3F74A8D863787C
:10542000002B0CD101218C4B19708D4B1A78002A5E
:105430005BD08C4B307801F0B9FE002855D00722A4
:10544000854B1A7051E061780029F8D1E378002B80
:1054500011D0854A854B1278307801F0A7FE607034
:105460006378002BEBD1200006F072F98020000257
:10547000684009B0F0BD784B1B78022BF3D00121B6
:10548000307806F07DF90028EAD10121307806F065
:1054900017FBE5E76378002BD1D16F4F032807D1C5
:1054A0003B78052B02D101333B701EE00223FBE762
:1054B0006F4B1A886F4B0293002A0BD01B78002B7E
:1054C00003D00121307806F063F93B78062B04D134
:1054D000013BE9E7029B1A70F7E7042B41D1012158
:1054E000029B3078197006F0EBFA5C4B1B68002BBE
:1054F000B9D01B68002BB6D0574A107884E7637880
:10550000554F002B27D10622211D5B4806F0E0FAFB
:1055100062895A4B5A491A80A2895A4B1A80E389E8
:105520000B800521397058490A80584A1380228A15
:10553000574B1A80574B1B78012B09D11F2001F0C4
:1055400047F8FA22920042430421307806F020F90D
:105550000022484B75E7312B00D070E70022454B05
:105560001A700323A0E706220021434806F048FBF7
:105570000023454A04211380444A30781380444A6A
:10558000138006F03DFA0821307806F039FAA37945
:10559000083B5A425341304A03331370304B1B7857
:1055A000002B06D0334B30781A78002A06D001F051
:1055B0003BFE0122314B52421A8096E701211970BD
:1055C00006F07EFAF5E70821307806F019FA6378DC
:1055D000002B00D047E72C4B2D4F0293E388029A13
:1055E00004211380294B307803932389039A138075
:1055F00063893B8006F0C4F8002800D033E7264BCF
:105600001B68002B00D12EE7039902983A8809887D
:1056100000881B68984726E74379132B00D022E7C0
:105620000389012B0AD11D4B1B78022B06D10821BF
:10563000307806F0E5F9FFF72BFE14E7052000F0BF
:10564000C7FF08210200307806F0A2F80BE7C04639
:105650001666FF1F051400001566FF1FAC65FF1FCF
:105660003644FF1F1744FF1FE865FF1FC965FF1F72
:10567000EA65FF1FEC65FF1FBB65FF1F0E44FF1FA0
:10568000C265FF1FC465FF1FB665FF1FB465FF1F1E
:10569000B265FF1FBA65FF1FA865FF1FB065FF1F3A
:1056A0008020C001014200D0E2E6CB0731D5324B69
:1056B0001B78002B1DD0314E05AC3378052B1AD149
:1056C000023B23702E4B21001B7823722D4B1B783D
:1056D00063722D4B187801F00DFD002809D00720CA
:1056E0002A4B30701B68002B03D01B68002B00D0A6
:1056F00098470120BCE60E20254B06221B78254941
:105700002370254B1B78637002ABC01806F0E0F9DC
:10571000D8E7022308001840194209D0174B1B781C
:10572000052B03D11D4B188806F07AF902209FE65D
:105730000424214203D0FFF737FD200098E6082318
:1057400008001840194200D193E6154B1C78012C33
:1057500003D0022C0DD008208AE6124B124A1349BE
:1057600013481B881288098800880094FFF7E0FD21
:10577000F1E7FFF78DFDEEE7EC65FF1F1566FF1FF4
:105780001044FF1FC665FF1F1666FF1FAC65FF1F95
:10579000C865FF1F1144FF1FC765FF1F0E44FF1F91
:1057A000B065FF1F0844FF1FB865FF1F0A44FF1FB5
:1057B0000C44FF1F10B502A804880B20002C10D148
:1057C000496808784978090201430C48814209D1A7
:1057D000022119800A4B59881170DB7800205BB2D6
:1057E000537010BD074C0A20A142FAD10221198042
:1057F000034B998811705B79F0E7C0466E2A000070
:10580000B063FF1F6F2A0000F7B5150008AA1688BD
:105810004A680F4F14785278120222430A24BA427F
:1058200014D10122DBB2019200962A0005F0A8FEF5
:10583000041E0BD1074B1B68002B07D068782A7811
:105840000002104342425041013098472000FEBD03
:10585000022900002866FF1F30B5012503790400E6
:10586000BFB02B4227D01549408805F0F5F92842F2
:105870000DD06A46124B69465B8D1380022353801C
:10588000104B5B8893806088002202F0C5FA0E49B5
:10589000608805F0E1F9C0070DD56A460B4B6946F3
:1058A0001B88138002235380064B9B88938060885B
:1058B000002202F0B1FA3FB030BDC0462066FF1FA3
:1058C0003844FF1FB063FF1F1866FF1F9244FF1F7D
:1058D00010B5074C0749200005F074F9200006496F
:1058E00005F070F90721054A054805F02DF910BDAE
:1058F000FFFF00002066FF1F1866FF1FD8BE0011C3
:105900003844FF1F10B5024803F008F910BDC04627
:105910005958001170B55F25082607498400CA78D8
:105920008B7840012A40B3433440A84323430243C9
:105930008B70CA7070BDC046A944FF1F010043B2FE
:1059400004205A0002409B000C3003401A431523E8
:1059500010B5044CE0789843143B0B4018430243C5
:10596000E27010BDA944FF1F10B5054B082419793A
:105970000A00A243002801D022000A431A7110BD78
:10598000A944FF1F10B5054B4024D9780A00A24353
:10599000002801D022000A43DA7010BDA944FF1F7D
:1059A0000821F8B5324D334BAE7804000E40AE708E
:1059B000984204DD67232B70473B6B70F8BD2E4B7C
:1059C000984203DAE0232B703A3BF6E700232B7072
:1059D0006B7083B21A0029485F3292B2284F82421C
:1059E0002CD9002C03DA5B421CB204232B70053443
:1059F00020B20A2106F034F804B2FA239B009C423C
:105A000032DB08232A7813432B706421200006F030
:105A100027F80A2100B206F033F809B22A787B5C35
:105A200013432B700A21200006F01AF80A2100B255
:105A300006F026F809B27B5C6A780AE06970002CEF
:105A4000DBDA5B421CB204232B70F3226B78092C47
:105A5000E8DC13436B700A21200006F011F809B24C
:105A60007B5C1E43AE70A9E7632CCEDCEDE7C0463D
:105A7000A944FF1F1B4E00001DFCFFFF2A08000069
:105A800002BF00110823F7B5194FCD003E7904007D
:105A90001E403E71EDB2632806DD5F3333433B7138
:105AA00020231D437D71F7BD0300093305DA202350
:105AB0005B4233433B71A623F3E70E4B019300286F
:105AC0000BDA0423444224B23B710A21200005F082
:105AD000D7FF019B09B25B5CE3E70928F5DD0A21EA
:105AE00005F0BEFF019B00B21B5C1E433E71ECE75C
:105AF000A944FF1F02BF001170B50F4B1B78002B8C
:105B000018D00E4E0E4D06223100280006F0A8F8DF
:105B100000280FD0062231000A4C280005F0D8FFDB
:105B20000120FEF7B3FC072221003E20FEF7DCFD3A
:105B3000FEF720FD70BDC0463366FF1FA944FF1F5E
:105B40002D66FF1F2C66FF1FE622402110B50A4B71
:105B50001A70403A5A703E329A70DA780A40DA7017
:105B6000082219791140053A0A431A71B5225A716F
:105B7000FFF7C2FF10BDC046A944FF1F10B5164C69
:105B80000A210223E05E05F06BFF00B2FFF708FF79
:105B90000423E05E642105F063FF012100B2FFF7FA
:105BA00071FF237A0024132220009A426041C0B280
:105BB000FFF7E8FE0320FFF7ADFE2000FFF7BEFE73
:105BC000064B1878053843425841C0B2FFF7CCFE67
:105BD000FFF792FF10BDC046B063FF1F1566FF1FA1
:105BE00010B5002801D0FFF7C9FF10BD002010B587
:105BF000FEF74CFC10223E200549FEF775FD002300
:105C0000984200D13E33034A1370FEF7B3FC10BD37
:105C1000F2BE00113366FF1F0200F0B501270A48EB
:105C20000A4E51188B1A002B00DCF0BD08241578A1
:105C30004308684038404000805B013C58406D0894
:105C4000002CF5D10132EDE7FFFF000012BF00117B
:105C5000F0B500250F269D4200DBF0BD4C5D070925
:105C600044403440A400A05801357840F3E70000D8
:105C7000F0B589B06A460D000B000F2711001035F2
:105C80001C780133260024093E40167054700232FD
:105C9000AB42F5D12023024AFFF7DAFF09B0F0BD8D
:105CA00018BF0011F0B54E780B7889B036020C00A1
:105CB000170001901E43012A61D9954B9E4200D8DE
:105CC00077E001339E421CD1062A17D1CA788B781F
:105CD00012021A430B791B0413434A7912061A4322
:105CE0008C4B5A6100221A705A808B4A5A608B4A38
:105CF0009A608B4ADA60002009B0F0BD8822520514
:105D0000EEE7884B9E423CD182498B78002B00D035
:105D1000F6E00C2A31D10F22A3789343E2781202E5
:105D200013432279120413436279120613434B6022
:105D3000E279A07912020243207A00041043627AC9
:105D400012060243CA60E27AA07A1202024376483F
:105D50004A81834208D804236E49142201980B70AB
:105D600005F0B6FE1420C7E71201D21889235B059F
:105D70009A42F0D801238B70BDE7022AFAD005239E
:105D8000EAE76A4A01239642E6D1FFF781FA052F36
:105D90000CD9E378A2781B021343227912041A4328
:105DA00063791B061343624A0393136005F018FEE0
:105DB000A1E7584D2B78002B9DD1AB78002B00D15B
:105DC000A0E02B8901339BB20093B34200D091E055
:105DD000132AD4D9CF7C8B7C3F02122120001F4391
:105DE000FFF71AFF874200D08EE0002E3DD1E37806
:105DF000A2781B0213432279E96812041A436379DB
:105E00001B06134303930A228B4212D1FF23A37074
:105E1000E370237163716B89002B09D1E37B227CD2
:105E20001B0212041343A27B13431B0901336B8132
:105E300000226B89002B8ED0002A67D16868370159
:105E40003818000B6B6900030390984205D968610C
:105E500005F006FDEB780133EB7068681022A11C99
:105E6000381805F025FD2E8145E76F89009A7B1EC5
:105E70009BB293423AD1E278A37812021A43237973
:105E800005A81B04134362796C6812061A43EB6879
:105E900000920392211D0C22049305F019FE0120AB
:105EA000260004A940421036FFF7E2FE013F012F11
:105EB00017D1009A0B232861824200D04CE70422BC
:105EC0001C49200005F0F4FC042203A9686805F0D1
:105ED00037FCE968039AFF23914200D13CE7F73B86
:105EE0003AE73100FFF7C4FE1036DFE70923B74277
:105EF000A4D831E7009BB34200D9FCE607232BE787
:105F0000022329E7032327E7062325E70A2323E7BC
:105F1000FFFE0000B044FF1F00000111FFFF000062
:105F20005048593601FF0000FFFF001102FF00003A
:105F300034F00040BC44FF1F10B5034C0B0001229D
:105F4000210000F06BFA10BDF96000110B8870B5EC
:105F500006000D000224162B11D92B00032209493B
:105F600000F05CFA041E0AD1074B2A881B88191C12
:105F7000934200D9111C300089B200F0EFFA2000E2
:105F800070BDC046256100118E66FF1F10B54A78AE
:105F90000400013A0B000220012A07D80A78002ADF
:105FA00004D005222000024900F038FA10BDC04696
:105FB000536100110A7810B50B0004000220002A7A
:105FC00004D007222000024900F028FA10BDC04684
:105FD000FF6100110A7810B50B0004000220002AAE
:105FE00004D009222000024900F018FA10BDC04672
:105FF0006562001110B5034C0B000B22210000F06C
:106000000DFA10BD9562001110B5034C0B000D2266
:10601000210000F003FA10BD0763001110B5034C16
:106020000B000F22210000F0F9F910BD616300118F
:106030000A7810B50B0004000220002A04D01122B7
:106040002000024900F0EAF910BDC046716300115A
:10605000002310B51322190000F0E0F910BD000074
:1060600010B5034C0B001722210000F0D7F910BD2A
:10607000C3630011002310B51922190000F0CEF9F6
:1060800010BD000010B5034C0B001B22210000F0D6
:10609000C5F910BDFD630011F7B584890D00060038
:1060A0000121002C22D000238268D3561778002BC0
:1060B0001EDA0C2C1AD90C3CA4B213194088009398
:1060C000230002F086FE431E984101307B06DB0F61
:1060D0006B703F23013C1F40A4B22870AF70AC80AE
:1060E000002C07D0B3680133AB6000210800FEBD6F
:1060F0000020EBE7AC60F8E70B7803704B88437047
:106100004B881B0A83700B79C370042070470420EE
:10611000022B06D10020537811781B02009A0B4302
:10612000138070470B8803700B881B0A4370022092
:1061300070470420009983420AD1537810781B02DB
:1061400003430B80D37890781B02034300204B80DD
:106150007047F8B50D004B7801240021461C0370F0
:106160002B788B4201D82000F8BD6B78B01C4F1CF7
:10617000012B10D1890069184B88022233704B889B
:10618000B9001B0A7370691805F052FD0436043417
:10619000A4B2F9B2E4E7122359436B185A880431C8
:1061A00032705B8810221B0A7370691805F040FD7D
:1061B00012361234ECE770B5049D14001E00052B56
:1061C00001D8042070BD637812781B0213432B8022
:1061D000E378A2781B02134302226B802A71211DEF
:1061E000681D063E05F024FDB2B22A81F02AE8D8E7
:1061F0002800A11D0A3005F01BFD0020E2E7002366
:1062000010B50A789A4201D8900010BD9A008A18F9
:106210005488013304705488DBB2240A4470948893
:1062200084709288120AC2700430EAE710B5110037
:10623000029C062B04D004201022142B01D010BD88
:10624000022222714B7808781B0203432380CB780B
:1062500088781B02034363800431601D05F0E8FC6D
:106260000020ECE710B50C788B7804315C43E4B285
:1062700003702200013005F0DBFC601C10BD04201F
:10628000022B06D10020537811781B02009A0B4391
:106290001380704710B50C000A88023105F0C8FC65
:1062A000208810BD70B504000D0004981100012B6A
:1062B00001D8042070BD1678527812023243028051
:1062C0000200F83255701470E825002C00D10C350E
:1062D000023B9AB24280AA42EBD80231043005F068
:1062E000A7FC0020E6E70420009983420AD15378F6
:1062F00010781B0203430B80D37890781B02034372
:1063000000204B80704710B50C000A88023105F060
:106310008FFC208810BD000070B501211E000420F4
:10632000049C0E400B4218D1CB40DDB28D4214D9F3
:106330000A49DBB2098899420FD32300F6331D7056
:106340003300580011184978165C090231430133B3
:106350002152D9B28D42F4D8002070BDD044FF1F25
:1063600010B50C000A88023105F062FC208810BDCF
:1063700010B50C788B7804315C43E4B203702200D2
:10638000013005F055FC601C10BD10B511000298DD
:10639000032B01D8042010BD14785278043B12025C
:1063A00022430280CA788C781202224342809AB239
:1063B0008280F22AEED80431063005F039FC002044
:1063C000E9E710B50C000B8803700B881B0A4370BB
:1063D0004B8883704B881B0AC3708A88043006314F
:1063E00005F026FCA088043080B210BD0420012BEB
:1063F00003D100201378009A1370704710B50C0079
:106400000B8803700B881B0A43704A8802300431E2
:1064100005F00EFC6088023080B210BDF0B589B086
:1064200003931E4B029242000700D05A019102F0E2
:1064300020F81325061E2DD0029B01240370019B1A
:10644000002B04D0001903999847001984B26B46B9
:106450001B7A5BB2002B0FDA1021380002F01CFB14
:106460001925002813D130003219E1B202F066FC80
:10647000051E0CD10C34A4B2042304AA380005A9CB
:1064800093800696948101F0AFFD051E02D0300086
:1064900005F04EF9280009B0F0BDC0468C66FF1F1C
:1064A00070B505000C0000280CD00020814209D0F6
:1064B00010222000044905F0BBFB01202B78237338
:1064C0006B78637370BDC04658BF0011F0B506000D
:1064D0000D0017001C0085B002291BD000201029D8
:1064E00007D1022B07D0102B03D115E00020102C70
:1064F00008D005B0F0BD69463800FFF7D1FF2A008B
:1065000069460BE069463000FFF7CAFF2200694682
:10651000380004E0022BE9D12A003900300005F0F0
:106520001FFBE6E7031CF72800D9F72303200849DF
:106530009AB2013A0B80D317034006499B189B106F
:106540000B80D30F04499B185B100B807047C0462B
:10655000D444FF1FD244FF1FD044FF1F034B1B88AE
:106560008B4202D3024B4000C1527047D444FF1FFC
:106570008C66FF1F014B4000185A70478C66FF1F46
:106580001722014B1A8070478C66FF1F70B50500FB
:106590000E2005F0EDF9041E13D0D0230370002364
:1065A0000622837007494570033005F041FB064B16
:1065B0002100DA8A62811B7E2373044B187805F070
:1065C000CFF870BDA866FF1F9866FF1F2445FF1F08
:1065D000262803D8024B4000C05A70470148FCE708
:1065E000D644FF1FFFFF000070B506000C00094DE8
:1065F0001C220021280005F003FB074B1E70074BEF
:106600001C7005F09DF90123002801D00023122001
:106610002B7070BD9866FF1F2445FF1FB966FF1FD2
:1066200070B505000D4C0800E260A1601022002149
:10663000656005F045FB012803D11021A06802F038
:1066400058FD10220021280005F03AFB012803D153
:106650001021606802F04DFD70BDC0469866FF1FB6
:1066600070B5041E05D1002903D006220D4805F09F
:10667000DFFA0D4B1D78012D11D1002C05D102221E
:106680001A7005F055FB280070BD00221A70074BE8
:106690001B78FF2BF7D02000FFF778FFF3E70025EA
:1066A000F1E7C046A866FF1F9866FF1F2445FF1F3D
:1066B000030010B5002801D1002010BD00780B4A5E
:1066C000002803D15988D1821B7913761378022BC5
:1066D000F2D10023984200D103331370044B1B788E
:1066E000FF2B01D0FFF752FF0120E6E79866FF1F5E
:1066F0002445FF1F002911D000280CD04B79012818
:1067000003D140225242134303E03F2213400328A7
:1067100002D001204B7170474022F4E70800FAE7ED
:1067200070B5094D0100287800280BD0074C0622CF
:10673000200005F07DFA21002878FFF7DBFF20001C
:1067400004F0BEFF70BDC046B866FF1F9266FF1F13
:1067500000290AD0012808D13F224B799343C02B4E
:1067600003D0403B5A425341981C704770B5174DB7
:1067700006002B78FF2B15D00A2005F0F9F8041E2F
:1067800010D0D0230370C83B8370114B11491B7884
:106790004670C3700622043005F04AFA21002878BA
:1067A00004F0DEFF0C4B1B78012B0DD10B4B1B684B
:1067B000002B03D09B68002B00D09847084B042186
:1067C0001878084A05F06CFA70BDC0462445FF1FD2
:1067D000B866FF1F9266FF1FB466FF1FE066FF1FCB
:1067E000E466FF1F60EA0000014B98687047C046EE
:1067F0009866FF1F014BDB68186870479866FF1F9B
:10680000074B10B5DA68136801331360054B18782D
:10681000FF2803D08021C90105F052F910BDC04600
:106820009866FF1F2445FF1FF7B50E0002F0C8F859
:10683000051E1CD00E4B06621F78002F00D1077872
:10684000AB791020019305F093F8041E0FD0D023EC
:106850000380C73B8370019BE91DC370062204308F
:1068600005F0E6F921003800E66004F079FFF7BD95
:106870002245FF1F014B18787047C046B866FF1FBE
:10688000054B002805D1054B1A78054B002A00D18D
:10689000014B18007047C046A866FF1FB866FF1F6F
:1068A0009266FF1F014B58687047C0469866FF1FED
:1068B000024B1868431E9841C0B27047BC66FF1F68
:1068C000421E03000120152A03D9FF3B5A425341BF
:1068D000D8B27047F0B51C0000230E0085B00390BD
:1068E00002920B70029A934201D3002019E0E55CFA
:1068F0005A1CD2B2002DF8D0029851198142F4DC12
:106900000233DFB2A35C18000193FFF7D9FF002820
:1069100007D0013D019A0399EBB233708A4202D14C
:10692000E01905B0F0BDDB19DBB2DBE710B50C00F8
:1069300002F09EF803001220002B03D0210058889B
:1069400005F0C6F910BD000070B50E4D8400635906
:10695000002B15D0186A002801D004F021FF2B5914
:10696000586A002801D004F01BFF2B59986A0028B0
:1069700001D004F015FF285904F012FF00232B5119
:1069800070BDC046C866FF1F1C4B70B504000E00EA
:10699000150099420AD11A4B1B68002B01D1122015
:1069A00070BD1B68002BFAD09847F9E7154B994248
:1069B00015D1134B1B68002B0AD01B68002B07D086
:1069C0009847002804D1104B1C70104B1D70E7E74E
:1069D00029002000FFF7AAFF0028E1D1F3E7080013
:1069E00001F0EEFF0028DAD003780320A342D7D1CC
:1069F0002900300005F06CF9D2E7C046FEFF000028
:106A0000C466FF1FFFFF0000C166FF1FC066FF1FB7
:106A1000F7B50400808801F0D3FF0025A84203D019
:106A20000578A08802F008F81C4E3378002B1FD0A0
:106A3000AB421DD11A4B28001978FFF777FF0028C9
:106A400018D000233370A3790820A778A688019373
:106A500004F08EFF011E0DD0D0230370CA3B83705B
:106A6000019B477086808371280004F079FE01E065
:106A7000002DE8D1A0880B4B8200D358002B01D009
:106A8000FFF762FF1721A088FFF768FDA08801F0DB
:106A900027FDA08801F0FEFDF7BDC046C166FF1FBF
:106AA000C066FF1FC866FF1FF0B587B01D000CABA6
:106AB0001B88070001930DAB1B88142002930EABBB
:106AC0001B88160003930FAB1B880091049310AB37
:106AD0001B88059304F04CFF041E1AD0D0230370CA
:106AE000CB3B47708370C670062229000430002D0E
:106AF00011D005F09DF8019B21006381029B009855
:106B0000A381039BE381049B2382059BA37404F070
:106B100027FE07B0F0BD05F073F8ECE7F7B500937A
:106B200008AB1B8807000C200D001600019304F031
:106B30001FFF041E13D0280001F042FF00280FD0D1
:106B40000078D0232370C93BA370009B21002381D0
:106B5000019B6770A580E680638104F001FEF7BDAC
:106B6000014B1878EDE7C0462445FF1F13B504001C
:106B700064890389C2888188C0780094FFF7CEFFBA
:106B800013BD000010B5044C2068002803D004F0A9
:106B900007FE0023236010BDCC66FF1FA122F0B5C5
:106BA000818892004A43384B384F1B6804009B1879
:106BB0009D2292009B18827989B01A603B68002B55
:106BC0005FD01D78324B1B68002B04D05B68002B14
:106BD00001D000209847260008363100E079FFF701
:106BE000B7FD237DE0710200E0780493638A2900F9
:106BF0000393238A0293E3890193A38800933300CC
:106C0000FFF752FFE378002B0BD1E289A379A1882B
:106C100002920196E27928000092012201F0DAFE48
:106C2000E0703B68002B20D0FFF7ACFF194D2878AF
:106C300000281AD0184B1978FFF778FE002814D0D6
:106C40002B78E67808200793A78804F091FE011EB0
:106C500009D0D0230370CA3B467083708780867149
:106C6000079804F07DFD00232B701721A088FFF703
:106C700075FCA08801F034FCA08801F00BFD09B080
:106C8000F0BD064B9DE7C0463409FF1FCC66FF1FD1
:106C9000E066FF1FC166FF1FC066FF1F2445FF1F80
:106CA000F8B5070008000E0001F08AFE041E18D097
:106CB0002620FFF78DFC051E00D12578062004F064
:106CC00057FE041E0DD00021062204F099FFD023A8
:106CD0002370C23B21006770A370A680E8B204F065
:106CE0003FFDF8BDF0B585B001930AAB1B780700F6
:106CF00002930BAB1B7808000D000092039301F088
:106D00005FFE061E22D0102004F032FE041E1DD0AD
:106D10001022002104F074FF2620FFF759FC002800
:106D200000D13078D0232370C13BA370009B210099
:106D30002372019B67706372029BA580A372039B01
:106D4000C0B2E3720C9BE36004F00AFD05B0F0BD35
:106D5000F7B50D00019001F033FE071E20D00E2084
:106D600004F006FE041E1BD02620FFF731FC061E91
:106D700000D13E78D0232380C53B0622A370F91DA5
:106D8000E01C04F055FF019B2A0063810123DD40D4
:106D90001A401D40210022736573F0B204F0E0FC3C
:106DA000F7BD0000F0B585B0029010000D0017008F
:106DB0000A9E039301F004FE041E31D0029B002BB7
:106DC0002ED1039B02795B0724D51223134304229F
:106DD000002E08D10B99002905D10C99002902D168
:106DE0000D9900291AD01A430D9B2271002B00D057
:106DF000C9E0002E00D1CFE0002D00D0CCE0606AC9
:106E0000002801D004F0CCFC1C21300004F040FF2D
:106E1000606205E002239A430E33D7E79343237160
:106E2000654BBA00D458002C00D1AAE0002E10D037
:106E3000236A002B03D11C2004F0DAFC20625E4B95
:106E4000BA00D358186A002803D01C22310004F07D
:106E5000EFFE0C9B002B12D0574CBB001D596B6AE8
:106E6000002B03D1162004F0C3FC6862BB00E3587A
:106E7000586A002803D016220C9904F0D9FE0D9B05
:106E8000002B11D04C4DBC006659B36A002B03D1C6
:106E9000142004F0ADFCB0622B59986A002803D08E
:106EA00014220D9904F0C4FE380001F089FD051E7E
:106EB00067D0414BBA00D358002B62D01A6A3420F5
:106EC000002A00D11C389A6A002A01D0143080B2FE
:106ED0000B9A002A01D01C3080B25B6A002B01D0D3
:106EE000163080B204F044FD041E4AD0182200215E
:106EF00004F086FE2620FFF76BFB0190002801D1ED
:106F00002B780193D0232370029B200063700A2307
:106F1000294EA370039BBD00A371AB59A780196ACA
:106F20001830002905D01C22A06004F081FE20004A
:106F300034307359996A002907D00300142214339E
:106F4000E060029304F074FE02980B9B002B08D0C3
:106F500003001C221C330B992061029304F068FE8D
:106F600002987359596A002903D01622606104F00F
:106F70005FFE6B462100187904F0F2FB3800FFF742
:106F8000E3FC05B0F0BD10220D9B0D991B69A01804
:106F9000236204F04DFE2CE70B9B002B00D13FE752
:106FA000012D00D03CE7606A002801D004F0F8FB16
:106FB0001C210B982AE7C046C866FF1F10B5044C79
:106FC0002068002803D004F0EBFB0023236010BDF1
:106FD000BC66FF1F0B4B07B51A68002A01D10020C1
:106FE0000EBD6946531C012012780731FFF772FC71
:106FF0000028F4D002780123100018401A42EED085
:10700000EEE7C046D866FF1FF0B51F4F01203B6872
:1070100087B0002B25D09B78059300F0B3FB0028A8
:1070200021D00A20FFF7D4FA04000B20FFF7D0FA92
:10703000164B05001E78731E9E413B68F6B2191D63
:10704000D878FFF757FB3B682900DA7A04330392BC
:107050009A7901930292009033002000059A04F07F
:107060001FFC07B0F0BDFFF7B5FF002805D00620D4
:10707000FFF7AEFA04000720D8E70820FFF7A8FAC8
:1070800004000920D2E7C046BC66FF1FB866FF1F98
:1070900070B50A4E040033780D00FF2B0DD004208C
:1070A00004F066FC011E08D0D0230370CE3B45706F
:1070B0008370C470307804F053FB70BD3445FF1FFB
:1070C00070B5040006200D0004F052FC011E0AD029
:1070D000D0230370CD3B8370054B44701B688580C3
:1070E000187804F03DFB002C01D0FFF767FF70BD5E
:1070F000BC66FF1FF8B5264F06003B680D00112443
:10710000002B05D10522234B1B78134202D11224F8
:107110002000F8BD204A10241268002AF8D0127806
:10712000002AF5D0DB0719D52B789A1E012A1AD828
:107130000C2004F05DFB132438600028E8D0002305
:107140000A22437029000670023004F071FDFFF737
:107150005BFF041E0AD0FFF731FFD9E700F012FBF6
:107160000028E1D1E4E7002BE2D0D0E70B4B1B78FD
:10717000032BCDD11D20FFF72BFA094B18800028D7
:10718000C6D0084B04211878074A04F089FDBFE7F0
:10719000BC66FF1FB966FF1FD866FF1FB866FF1FDA
:1071A000B666FF1FE466FF1F60EA0000F7B50193B3
:1071B000194B14001A78052306000F0012201A42FA
:1071C00021D0012920D1154B1D68002D1BD0022094
:1071D0001F2C18D8002C02D0019B002B13D0104B71
:1071E0001F221E706E1C0021300004F009FD019961
:1071F0002200300004F01CFD310020002C70002F14
:1072000006D004F07DFDFEBD064B12201D68DCE7B4
:1072100004F0EEFCF7E7C046B966FF1FD866FF1F13
:107220003445FF1FD466FF1FF8B50F4E1224336894
:10723000002B17D01B780F3C834213D100250B4F36
:107240000221387804F0DCFB094B042138781D80DA
:1072500004F0D6FB074B28001D8033685C7004F0F7
:10726000EFFA04002000F8BDBC66FF1FE466FF1FB4
:10727000D066FF1FB666FF1F70B5012823D11B4CD7
:107280002388002B03D01A4A1578002D07D0194BFC
:107290001B68002B02D01878FFF7C6FF70BD3B2B90
:1072A00002D93C3B2380F9E7134E0221307804F0E9
:1072B000A7FBFA222388920002215A43307804F077
:1072C00067FA2580EAE70B4B1B68002BE6D00B4BD7
:1072D0001B785B07E2D5084B0221187804F090FB7D
:1072E0000022024B1A80FFF769FED7E7D066FF1F26
:1072F000B466FF1FBC66FF1FE466FF1FB966FF1F71
:10730000F8B51E4D2868002803D004F049FA002380
:107310002B601B4E3068002803D004F041FA002394
:107320003360184F05243B7818002040234221D0B9
:10733000154800F02BFA3B78234213D0202004F0AC
:1073400057FA2860002813D02022002104F058FCAE
:10735000202004F04DFA041E306005D020220021C8
:1073600004F04EFC002004E0286804F019FA2C60B8
:107370001320F8BD00F00AFAF4E7C046D866FF1FF4
:10738000D466FF1FB966FF1F2845FF1F10B50A4CC2
:1073900023681A1E0ED0002808D10130587004F05E
:1073A0004FFA002805D02368002B02D00021FFF7F8
:1073B00087FE0122100010BDBC66FF1FF7B5274EE7
:1073C000050033680191181E21D05C78244F012CF0
:1073D00030D1FFF7FFFD002825D02000FFF7F8F897
:1073E0000400412814D91F4B022118781E4A04F0CA
:1073F00057FC1E4B3C3C1C80022233685A703B7881
:10740000002B14D128000199FFF75AFE0120FEBD80
:10741000FA2292004243002AEED0124B0221187841
:1074200004F0B6F9E8E7FFF7D3F80200F3E700232A
:107430003B70EBE73B78002BE8D1032004F098FA8F
:10744000011E08D0D0230370CC3B45708370336895
:10745000187804F085F9FFF7B1FDD7E7BC66FF1F88
:10746000B466FF1FE466FF1F60EA0000D066FF1FDE
:1074700010B51749838802008B4220D011D81549D6
:107480008B4217D0144900205B1899B2012907D804
:10749000926811785A425341D8B2FFF7F9FD0120A2
:1074A00010BD0E4A00209B1807229BB29A42404111
:1074B000C0B2F5E783681878FFF768FFF0E78368E4
:1074C00099785A78090218781143FFF777FFE7E7B0
:1074D0000A20000006200000F8DFFFFFAFDFFFFFFB
:1074E000014B18707047C0463545FF1F10B5064C5C
:1074F000207001F041FA207804F0FAF90521207893
:1075000000F062FD10BDC046E466FF1F0BB273B50C
:107510000D00002B00DBC4E0884B187804F040FB22
:10752000041E0ED00378912B0FD0A22B00D1A1E026
:10753000834B1878FF2852D0210004F011F900285D
:107540004DD180200002684076BD43780F2B76D065
:1075500013D8052B70D00E2BEAD18088794B984236
:107560002BD8794B98421BD8784B9842E0D1A3682E
:107570001878591CFFF774F838E03E2BD8D183787F
:10758000032B74D06CD8012B6ED0022BD0D1704B52
:107590001B68002B23D05B68002B20D098471EE08F
:1075A0006C4BC0180C28C3D804F0BAF81DC2C21521
:1075B0000BC20B0B0B3223C23C00674BC0180728D1
:1075C000B6D8664B1B68002B09D01B68002B06D071
:1075D000200098470AE0A3681878FFF7C7F8200052
:1075E00004F0B6F8ADE7A068FFF762F800289FD076
:1075F000F5E7A3681B78002BF1D0554B1B68002BD7
:10760000EDD01B68002BEAD0210055489847EDE7E4
:107610004F4B1B68002BE2D01B68002BDFD02100F2
:107620005048F3E7504B1B68002BD8D05B68002B09
:10763000D5D021004348E9E7FFF7EAF9CFE7808892
:107640004A4B984203D04A4B984200D070E7464BD1
:107650001B68002BC3D05B68002BC0D02100D5E78E
:10766000153B012BBBD963E7FFF798FAB7E7FFF7A4
:107670007DFAB4E73F4B1B78042B07D100236A4601
:1076800013800179408800F0C5FCA8E7364B1B68E1
:10769000002BA4D05B68002BA1D00100364898478E
:1076A0009DE7012421420AD0294B1B68002B04D0FE
:1076B0005B68002B01D000209847012043E78B072F
:1076C0000AD5264B1B68002B04D05B68002B01D029
:1076D00020009847022036E70421280008400D4288
:1076E00000D131E7254E3388002B21D0013B9BB2DE
:1076F0003380002B1AD1FFF7DBF800280AD0204B8B
:107700001C70164B1B68002B04D05B68002B01D04B
:1077100020009847FFF7C6F8694601F001FD68466A
:10772000FEF7FEFF1D20FEF753FF308004200AE71E
:10773000024B187804F064F9F8E7C046E466FF1FCE
:107740003545FF1F0E200000012000000910000039
:10775000DC66FF1FFEDFFFFFAFDFFFFFE066FF1FFE
:107760000C2000000B200000C466FF1F0D2000004D
:1077700013200000B966FF1FFFFF0000B666FF1F61
:10778000B466FF1F10B501F09BF910BD014B1860E6
:107790007047C046E066FF1F0B880020162B01D8FB
:1077A00017230420014A13807047C0468E66FF1FCE
:1077B00000207047074A03001188814207D0918852
:1077C0000020994202D1013080001018704700203B
:1077D000FAE7C046EC66FF1FF0B58F7806000D0093
:1077E000C7B01E2F15D1FFF7E5FF051E03D10024FA
:1077F000200047B0F0BD00223B003100C07800926D
:1078000000F0B2FB0400A81C00F0D3FBFF23EB70D8
:10781000EEE7264B062403931B78FF2BE8D0182FA6
:10782000E6D87B08224A013BDB0002929A58944634
:10783000002ADDD0029AD3185B68002BD8D00878D4
:10784000002802D14B78012B02D10624122FCFD170
:1078500007AFAB88697800976446AA68A047041E02
:10786000C6D1AB78029A5B08013BDB00D318390024
:1078700030005B689847041E0BD1AB78042BB6D060
:10788000039A310010782200009700F06DFB04008D
:10789000AEE76A78002AABD1AA7805A93B880871BF
:1078A00030000A704B80FEF747FBA0E73845FF1F0A
:1078B00068BF00111D4B37B5050098420BD0002959
:1078C0000AD1FFF777FF002805D11948FFF772FFAB
:1078D000002800D0058037BD01291AD1FFF76AFFC3
:1078E000041EF8D001235B420380A378FF2BF2D063
:1078F000FE2B07D00023E0781422009329001E33CA
:1079000000F032FBA01C00F054FB01235B426380BB
:10791000E1E70229DFD1013901F0BEF80028DAD110
:107920002800FFF747FF041EDFD1D4E7FEFF000069
:10793000FFFF0000022210B5074B52421A80074891
:1079400001325A809A80DA8000F07EFA044801F011
:1079500025F8002010BDC046EC66FF1FD977001146
:10796000B57800110388F7B50400002B02D1022579
:107970002800FEBD42680221137825485268FEF7B0
:10798000A5FD00282ED0234F01253A88002AEFD0EC
:10799000802321885B0201259B1A9942E8DC0C2098
:1079A00003F026FF061E31D03B8822889C46002328
:1079B0001800019561469DB2491989B2AA421BD8A7
:1079C000002801D062443A8000233000082208C019
:1079D000210004F02DF9104A1368002B13D1002563
:1079E0001660C5E76268022113780C485268FEF7FA
:1079F0006DFD0028C7D1BAE760681D0140194181BB
:107A000001330198D6E71A001B68E6E71325AFE7B4
:107A1000D6BF00113645FF1FE866FF1FD4BF001117
:107A2000014B18707047C0463845FF1F14230A00E9
:107A300010B51A40194204D00122102101F048F873
:107A400010BD4B06F9D4012088434000F8E710B57B
:107A500014008B0604D50122102101F039F810BD65
:107A600008230A001A40194202D14BB2002B0FDA48
:107A7000102101F02DF8002808D02300F9331B78DD
:107A8000002BECD0F8342378012BE8D10020E6E776
:107A900003208907FAD4E2E7F0B51F00184B85B040
:107AA0001C68019002910392002C27D1200005B0A0
:107AB000F0BDA5683301ED186B89019A934211D38B
:107AC000029A93420ED8002F04D10A9B002B10D1AA
:107AD0002C00EBE73B002978039A6868FEF7F6FC78
:107AE0000028F2D10136B6B2A388B342E1D82468A7
:107AF000DAE7A3680A9A5B891380E9E70026F3E7CF
:107B0000E866FF1F37B50C000A88498801239142B7
:107B100017D3002A15D0651D23792A0002210A48AF
:107B2000FEF7D4FC102300280BD02379618820882D
:107B300000242A000094FFF7AFFF0A23A04200D0E0
:107B4000230018003EBDC046D6BF001113B50A0081
:107B500008884988012388420BD8002809D00024CE
:107B6000137905320094FFF797FF0A23A04200D053
:107B70002300180016BD13B50A00088849880123A0
:107B800088420BD8002809D00024137905320094CC
:107B9000FFF782FF0A23A04200D02300180016BD81
:107BA000F0B58BB003904A8808880E00012382420A
:107BB00055D3002853D00023012704AC23700022A2
:107BC000718813000092FFF767FF051E3ED02078F2
:107BD000002835D12B78022B18D167706A89830071
:107BE0000130E31880005A8069680222201804F0EE
:107BF0001FF823780133DBB22370042B19D93B0023
:107C00006889013080B2002BD9D01FE00223637055
:107C1000122358436A89231804305A806968102255
:107C2000201804F005F823780133DBB22370002B11
:107C3000E5D10C4A6B899B185A425341DBB2DFE70E
:107C40006378012BE4D12B78022BC7D022780A234A
:107C5000002A04D021000398FEF798F900231800A9
:107C60000BB0F0BD0100FFFF0F4BF0B5040018682A
:107C7000002816D083685D89A54207D88288AE188F
:107C8000B44203DA12019A18934201D10068EFE777
:107C90001E005F891036A74204D1002900D00D8054
:107CA0001800F0BD3300EFE7E866FF1F70B5050070
:107CB0000C0008880021FFF7D7FF03000120002BEC
:107CC00004D022002800197AFFF7C1FE70BDF7B575
:107CD0000C00002501902300F6331B78AB4201D83D
:107CE00000200AE06B00E65A00213000E718FFF799
:107CF000BBFF002802D126800130FEBD017A019829
:107D0000FFF794FE002802D03B882380F5E7013579
:107D1000EDB2E0E710B5040008880021FFF7A4FFEA
:107D200003000120002B03D02000197AFFF77EFE0C
:107D300010BD0000054B1B68002B01D1180004E0AA
:107D40009A6852898242F6D198887047E866FF1F88
:107D5000F0B50E27002687B0039302ABFF183E80D4
:107D600005001F4B40891400984207D02B78013042
:107D700000976A6880B2FFF78FFE060002212B7819
:107D800018486A68FEF7A2FB00280FD06C89200013
:107D9000FFF7D0FF002802D0013C0419A4B2039BD6
:107DA000002B00D01C80300007B0F0BD02212B78E2
:107DB0000D486A68FEF78AFB0028E7D102212B787C
:107DC0000A486A68FEF782FB002807D0002EDED042
:107DD0003B88A342DBD17489013CDFE76C89DEE795
:107DE000FFFF0000D6BF0011D4BF0011D2BF0011A9
:107DF00010B50C00FFF7DEFC03000220002B0AD0B8
:107E0000002C00D023609B781720FE2B03D0013874
:107E1000FF2B00D1002010BD73B50D0001A9040097
:107E20001600FFF7E5FF172805D0002E04D1290022
:107E30002000FEF727F976BD01221021200000F076
:107E400047FE0028F3D0F6E7014B18607047C046A4
:107E5000F866FF1F37B56B469D1D01000400022226
:107E6000280003F035FE2B88B02B0ED12379122B7E
:107E700009D12300FF339B78012B06D101216088B3
:107E800000F0E0F801E01B2BF8D037BD10B5054B32
:107E90000421187000F098F8FFF74CFDFEF770FB16
:107EA00010BDC046FC66FF1F0020F0B50BB20F00EE
:107EB00087B0834234DA274B187803F071FE051E31
:107EC0002BD00378A02B25D103AE3100FEF7E4F8C8
:107ED000041E0BD1B378DB0724D51F4B06341B6877
:107EE000002B03D03100688898470400A868002858
:107EF00001D003F01DFC002C08D1184A039B13404D
:107F0000174A934206D0B3781B2B03D0012168880F
:107F100000F098F8280003F01BFC80200002784055
:107F200007B0F0BD0F4B1B68002B10D031006888E4
:107F30009847041EDAD07378002BD7D1B27801A904
:107F40000A704B800C716888FDF7F6FFCEE70624B7
:107F5000F1E7C046FC66FF1FF466FF1F00FFFF004D
:107F600000011200F866FF1FF7B501908220400063
:107F70000D0017001E0003F0FBFC04001320002C72
:107F800012D0B02320002370089BFC22677065800C
:107F900026710830002B08D0190003F049FE21009B
:107FA000019803F0DDFB0020FEBD089903F028FED8
:107FB000F5E710B5041E06D00078FD2803D803F0BD
:107FC00007FCFF23237010BD0A1F93B210B50400F5
:107FD0000220032B05D882400020024BD1529B186F
:107FE0009C7010BD1C67FF1F0B8870B5043B04001C
:107FF0000D000220032B0BD80121200000F04CFDC6
:1080000003001420002B03D02900200000F0DEFB29
:1080100070BD000007B51300034A00920A00012159
:1080200000F02CFC0EBDC0465182001107B5019234
:1080300003220092024B0A00122100F049FC0EBDFF
:10804000CF82001107B56B4601AA11800449D88080
:1080500008780633012802D1190003F0B9FD07BDE5
:10806000FD66FF1F0C4B10B518700023FF210B4A53
:108070001380138193819380094A53801370517246
:1080800093819372D174D3821375517703F0F0FB0F
:1080900000F0FCF910BDC0462C67FF1F1C67FF1FD6
:1080A000FE66FF1FF0B58DB06B46002003910C22D9
:1080B0009B5E834200DBB0E05D4B187803F070FDFF
:1080C000051E00D1A4E00378902B00D09DE006AF00
:1080D00001004688380000F013FA7968040000298E
:1080E00000D19CE03B88052B6ED13B89032B1CD92A
:1080F00005AC200000F0A2F86288172A61D83989FF
:10810000131D994231D17968237804310291D9073E
:1081100038D5607800F08EF9071E06D00023037171
:108120002378012B08D0132B23D0A868002800D176
:1081300078E003F0FDFA75E06288029909A800F082
:10814000A6F80290380000F08BF909AA2378387A53
:108150000192002231000092029A00F012F93800D8
:1081600000F064F9029B002BDFD0300000F080F9B2
:10817000DBE70378032BD8D16288029909A800F0C5
:10818000D6F8DEE7122B13D1029909A800F0B5F852
:10819000021EEAD127498B88002BC6D0887909A90D
:1081A0002378019161780091310000F0EAF8BCE792
:1081B000002302AA93833000617809AAFFF72AFFFF
:1081C000B3E71D4B0993F6E7042B02D09A1F012A4F
:1081D000ABD8184A043B9B00995A0029A5D0D21865
:1081E000907831003A0000F0AEF800289DD13B882D
:1081F000042B03D001213000FFF724FF012C04D110
:10820000A868002801D003F093FA280003F0A0FA30
:108210008020039B0002434018000DB0F0BD0128F0
:1082200000D182E701213000FFF70CFFEDE7C046E7
:108230002C67FF1F1C67FF1F010017000B780370DE
:108240004B784370CB788A781B0213434380704786
:108250000A88030002700A88120A42700A88012AFA
:1082600006D14A8882704A88120AC2700420704778
:1082700002208242FBD14A8804309A704A88120A4E
:10828000DA708A881A718A88120A5A71EFE710B573
:108290000400012082420CD94B780A781B02134358
:1082A0002380834206D1CB788A781B0213436380F4
:1082B000002010BD022BFBD1CB788A781B02134320
:1082C00063804B790A791B021343A380F0E70B8884
:1082D00003700B881B0A43704B8883704B881B0A02
:1082E000C3708B8803718B881B0A4371CB888371A1
:1082F000CB881B0AC3710820704703000120082A9D
:1083000014D14A780878120202431A80CA78887811
:10831000120202435A804A790879120202439A8073
:10832000CA798879120202430020DA80704710B5BA
:1083300004000120022A05D100204B780A781B0294
:108340001343238010BDF8B5060010200F00150060
:1083500003F00EFB04000120002C0ED0A0230C2201
:10836000290023806780201D002D07D003F060FCCA
:108370002100300003F0F4F90020F8BD03F040FCC8
:10838000F6E7F7B51E00009008AB142017001D7823
:10839000019103F0EDFA041E12D0A2230370019B99
:1083A00047704380099B057146710C220830002BF1
:1083B00007D0190003F03CFC2100009803F0D0F92D
:1083C000F7BD099903F01CFCF6E737B5041E0FD082
:1083D0004388002B0CD00025C1881323007A172274
:1083E00001950095FFF7CDFFFF236580637225702F
:1083F00037BD000010B50C4904004A88002A09D096
:108400008B89002B05D00020CB8A0222834201D029
:1084100010BD012213000A20434300204032C854FB
:10842000C81842800472F3E7FE66FF1F00234380F2
:1084300003707047094B00211A0010B55C88002CAE
:1084400006D01C79844203D10A234B43D01810BDB7
:1084500001310A330329F1D10020F8E7FE66FF1F3E
:1084600010B50400407A03F0B3F9FF23637210BD26
:108470007047043010B580B203F05AFA002803D0D8
:108480000421494203F09CF910BD000070B500259D
:10849000104CA0682580A581A580A84202D003F0D9
:1084A00047F9A56000250C4C0C4B606D1D80230026
:1084B00058331D70A84202D003F03AF965650025D3
:1084C0006068002801D003F033F9013508340A2D23
:1084D000F6D170BDC467FF1F6867FF1FB867FF1F35
:1084E00070B5041E09D1054D2880A881A880A86810
:1084F000002802D003F01CF9AC6070BDC467FF1FF8
:10850000F0B54B8885B00193002343600A790500DC
:108510000F00022A00D07BE0CA88032A17D98B6893
:108520005E7819783602DC78D8790E4399781B7A10
:1085300024021B020C43034353495BBA0B80331DD7
:1085400093421ED1042C04D0631F022B0ED90120AC
:1085500015E0019A4D4B1201D35A002B06D0019819
:10856000FFF7BEFF4A4A1369013313610421B8685B
:108570002E812C80494203F023F96860002005B069
:10858000F0BD434D042C06D0631F022B0FD9EB68BE
:108590000133EB60DBE7019A3C4B1201D35A002B0D
:1085A00005D00198FFF79CFF2B6901332B61374BF6
:1085B00030000293019B029A1B0101930023019951
:1085C0008C468B52130063449C8003939E81FFF77B
:1085D00050FF039B041E986016D00421B8684942DE
:1085E00003F0EEF8FA880100043A200003F020FBC3
:1085F0000199029AFB888A5A043B9B18029A8B5273
:108600002B6801332B60A2E7AB690133AB619EE7B6
:108610001E4B0293019B1E01029BF35A002B2DD08F
:1086200002998C19A068002828D0012A26D1FA883E
:108630009B189BB27352A189994217D39B1AC018F9
:10864000B96803F0F5FA029BA289F35A934200D06D
:108650007DE700222B81A3882B80A3686B60029B9F
:10866000F2520B4A53680133536070E7084A93682B
:10867000013393600198FFF733FF68E7044A5369B9
:1086800001335361F6E7C0462E67FF1FC467FF1F23
:108690003467FF1F70B5051E15D10B4C0B4B1880AE
:1086A000230058331870606D002802D003F040F8A2
:1086B0006565250050356068002801D003F038F862
:1086C0000834AC42F7D170BD6867FF1FB867FF1F61
:1086D000F0B51700A12285B0920001934243394BB7
:1086E00006001B680C009B18D933FF331D78FDF77B
:1086F00041FF0430854204DD3000FDF73BFF0430CC
:10870000C5B2BD4207D33A0000213000019B03F0FF
:1087100017FB05B0F0BD2900380003F031F9230044
:10872000C6B250331E700393019B29006365380065
:1087300002F0BEFFCBB20293002B02D0039B0136A6
:108740001E7000262300503303931B78B34204D8D5
:10875000606D002831D10020DBE7029A2800002A52
:1087600004D0013B1000B34200D02800F700E71905
:10877000387003F0C5F9786000280ED03A78019976
:1087800003F056FA019A3B780136D3180E4A01934A
:10879000D369F6B20133D361D4E7039B18706065E7
:1087A000A74205D1084A1320D36A0133D362B0E748
:1087B000606802F0BDFF0834F2E702F0B9FF002361
:1087C0006365C8E73409FF1F3467FF1FF7B50D0065
:1087D00007000421686802F0F3FF2B89040003708E
:1087E0002B891B0A43702B8883702B881B0AC3704C
:1087F0002E8902250436F6B2FB2E15D81B4B9F425C
:1088000014D10C2003F0B4F81135011E0CD09023C4
:1088100003708E3B0371043B4380154B8460C6801C
:10882000187802F09DFF00252800FEBD5C237B43E5
:10883000104AD3180093583301931B78002B0FD1A3
:108840000300320038000099FFF742FF019B05004A
:108850001B78002BE8D13800009903F029F9E3E7F1
:10886000054A0725536A01335362DDE7FEFF000026
:108870002C67FF1F6867FF1F3467FF1FF0B587B0C5
:10888000009017200F0016000193FFF7F2FD13254B
:10889000041E19D00C98031E02D00199201D984780
:1088A000030AE370052302AAA070043090812770A8
:1088B0000098667003A993800494FFF787FF051E54
:1088C00002D0200002F034FF280007B0F0BD000005
:1088D000F0B587B01F000CAB1B7803910593012105
:1088E0000DAB06001C78049200F0D6F81425002881
:1088F00021D02000FFF77EFD0135041E1BD0114959
:10890000059B0A7803700132D2B2131EC68001D1D2
:1089100001231A000B7022713000049B0399009709
:10892000FFF7ACFF051E09D1230021000648074AC6
:10893000093303F0BDF9280007B0F0BD00236380C0
:108940002370F8E73067FF1FCB83001130750000FC
:10895000F8B505000E00064C064F2368002B02D028
:108960003100280098470434BC42F6D1F8BDC04617
:10897000D467FF1FE867FF1F0123064A5B4253804D
:10898000002313715362044A136053609360D360F1
:1089900013617047E867FF1FD467FF1F02000023C1
:1089A00010B506499C000859002801D1625010BD3D
:1089B0000133052BF6D11320F9E7C046D467FF1F1A
:1089C000034A5388181A43425841404210407047A6
:1089D000E867FF1FF0B585B002930AAB1F780CABB8
:1089E0001B88009008000E0001920393FFF7E8FF38
:1089F00005001120002D1BD10E48FFF7E1FF0400F8
:108A00001520002C14D006220B99A771E01D03F04D
:108A10000FF9019B30002371029B29006371009BB9
:108A200066802370039B6562E381FFF791FF280056
:108A300005B0F0BDFFFF000010B5FFF7C1FF040057
:108A40000220002C12D060880121FFF781FF606AAC
:108A5000002801D002F0A4FE28220021200003F00B
:108A6000CFF8012300205B426380207110BD00001D
:108A700030B5074A074C5588010013780020A542FD
:108A800004D05B1A59424B415842104030BDC04699
:108A9000E867FF1FFFFF0000084A10B501230C0024
:108AA000904208D0FFF78CFF031E04D003792340C7
:108AB0005A1E9341DBB2180010BDC046FEFF0000F5
:108AC000024B1879431E9841C0B27047E867FF1FF8
:108AD00070B504000D001600FFF772FF002804D1E6
:108AE0000D4B9C4200D0143070BD416A03790520C3
:108AF000002907D012221A40102A02D10520002E88
:108B0000F2D10F20DB06EFD5897E0C20A9428941E6
:108B1000494249420840E7E7FEFF0000030010B564
:108B2000002800D110BD0348034A41889142F9D082
:108B30009847F7E7E867FF1FFFFF0000002330B505
:108B4000C45CCD5C6C40D4540133102BF8D130BDE3
:108B50000F23002210B5C45C64002243CA54C25CD7
:108B6000D209013BF7D210BD0200010010B520323E
:108B7000103102F02DFF10BDF0B58BB00390102026
:108B800005931700049102F033FE0090102002F0CC
:108B90002FFE009B13240190002B05D000280CD140
:108BA0001324009802F0FCFD019B002B02D018005A
:108BB00002F0F6FD20000BB0F0BD102002F018FE10
:108BC0000600102002F014FE13240500002E00D130
:108BD000AEE0002819D01022002103F011F8320075
:108BE0002900039802F0F4FE041E0ED133787F2B87
:108BF00051D830000099FFF7ABFF009B1B787F2B0B
:108C000053D801990098FFF7A3FF300002F0C8FD88
:108C1000002D02D0280002F0C3FD002CC1D110208D
:108C200002F0E6FD0600102002F0E2FD0290002EA8
:108C30007CD0002878D03A000F3223000125121191
:108C400005D00F333B4015B25A4253411BB26A1E46
:108C50001201002B33D0049BD2B298180099029ACB
:108C6000FFF76CFF013D10220021300002F0C8FF29
:108C7000ADB2049F2D017D19AF4242D0002C33D0FC
:108C8000300002F08DFD029B002B00D189E7180017
:108C900002F086FD85E729003000FFF759FF280024
:108CA0002549009AFFF74AFFA7E729000098FFF738
:108CB0004FFF28002049019AFFF740FFA5E70F2149
:108CC0000F4004998A18D9B28F4208D9D15C06A8FE
:108CD00019540133102BF6D1029A0199C0E7791A81
:108CE00048424141C901F2E73900300006AAFFF7C6
:108CF00025FF3200039806A902F06AFE103704002F
:108D0000BAE7002CBCD13000029906AAFFF716FF83
:108D1000320006A9039802F05BFE0822040031002D
:108D2000059802F085FFABE71324A9E71324AAE70F
:108D3000002800D06EE733E7DCBF0011F0B58BB040
:108D40000F0016000225009000283FD0002A3DD0D9
:108D50000B1DDBB21800029302F04AFD1135041E10
:108D600034D0FDF747FD05003A000099201D02F0C0
:108D70006FFDEBB20393E3702B0CDBB22F0A009371
:108D80006370FFB22B0E2370A7700193FDF72CFDCB
:108D90001022010006A802F05BFD2100029A04AB3C
:108DA00006A8FFF7E9FE051E0DD1039B08223370CC
:108DB000009B04A9B370019B7770F370301D02F023
:108DC00047FDFDF71DFD200002F0EAFC28000BB076
:108DD000F0BDF0B58FB00D00149E03900492059382
:108DE000002A03D1022420000FB0F0BD002EF9D0DC
:108DF0000398FFF7E5FD1424071EF4D0727833784A
:108E000012021A43B3781B041343F27812061A4372
:108E1000036A0192934201D30133E3D1002D03D0C1
:108E20003B7901249B07DED50822002106A802F029
:108E3000E7FE059B13240433DBB21800029302F013
:108E4000D7FC051ECFD0059A0499043002F000FD2E
:108E500004223100280002F0FBFC390010221031FE
:108E60000AA802F0F5FC2900029A06AB0AA8FFF74F
:108E700083FE041E0FD1082206A908A802F0E8FC10
:108E80000822311D08A802F06BFE012807D10199C4
:108E90000398FDF7C9FC280002F082FCA3E7012437
:108EA000F9E7000070B51C4C05002368181E10D0AF
:108EB000002D14D11A78002A0CD1981C083202F027
:108EC000B7FE02F045FE0135002808D123681D7069
:108ED000012070BD0A331800082202F0A9FE2368A1
:108EE000002BF5D0122002F043FD061E0DD0C12349
:108EF00021680370457002311022023002F098FEA2
:108F000023683100587802F02BFC206802F048FCFE
:108F100000232360DCE7C0461068FF1FF8B504009B
:108F20002020FDF755FB0D4EA700BB590500002B77
:108F30000DD000280BD0D878FF2809D108492A0085
:108F40000C55F35907480333611802F0B1FEF8BD20
:108F5000290002F06DFD0028F0D1F8E72C68FF1F12
:108F60001468FF1F75A1001170B5064D8400635988
:108F7000002B05D0D87802F02BFCFF226359DA7061
:108F800070BDC0462C68FF1F70B506008CB00C0089
:108F9000150000213022684602F032FE3100102216
:108FA000684602F055FC1D2021000322684402F0AF
:108FB0004FFC6846FFF7D8FD2D210400032228004E
:108FC000694402F045FC20000CB070BDF0B507000C
:108FD000160097B001931CAB1D7830221EAB009198
:108FE0000AA800211C7802F00BFE102239000AA802
:108FF00002F02EFC1022002102A802F001FE07223E
:10900000310002A802F024FC072202AB9818631E6C
:109010009C41019902F01CFC02AB9C732B005A1E70
:10902000934102AAD3730021102206A802F0E8FDA2
:1090300006221D9907A802F00BFC1A2002ABC018EB
:1090400006221F9902F004FC102200990EA802F0DB
:10905000FFFB102202AB0EA908781C78013A604091
:10906000D2B2087001330131002AF5D10AA8FFF706
:109070007BFD102212A904000EA802F0D9FD1022D7
:1090800006AB0EA908781D78013A6840D2B2087084
:1090900001330131002AF5D10AA8FFF765FD044329
:1090A00010222098E4B212A902F0D2FB200017B0DF
:1090B000F0BD70B50E0014008CB00100102268469F
:1090C0001D0002F0C5FB3100082204A802F0C0FB1D
:1090D0002100082206A802F0BBFB6846FFF744FD0A
:1090E00004001022280008A902F0B2FB20000CB0F6
:1090F00070BDF8B506000D0000243719AC4200D34E
:10910000F8BD02F06DFB030A3B70631CDBB2013754
:109110009D4203D90234F054E4B2EEE71C00EDE7BF
:1091200073B506000C000225002819D0002917D0BD
:10913000032101A8FFF7DDFF6B469A793F231A4010
:10914000013313436A463000937101A92200FFF7EF
:109150001BFF051E04D10322E01C01A902F068FDDB
:10916000280076BD03785807DA08C00FD2008000C7
:109170009B0710439B0F1843C0B2704707230B4057
:10918000C908C9000B4303707047000070B50400A4
:10919000FFF7EAFE134DA4006359002B21D0186A93
:1091A000002801D002F0FCFA2B59986E002801D05B
:1091B00002F0F6FA2B59D86E002801D002F0F0FA2E
:1091C0002B59186F002801D002F0EAFA2B59586F7A
:1091D000002801D002F0E4FA285902F0E1FA002355
:1091E0002B5170BD2C68FF1F0E4B8000C35870B50B
:1091F0000C00002B0FD09D68002D0CD02B78201D6B
:109200000B706B784B70A97CFFF7B8FF2B7E237235
:109210006B69E36070BD10220021200002F0F0FCB9
:10922000F8E7C0462C68FF1F014B18607047C04626
:109230002868FF1F074A03008000825810B5002AE3
:1092400006D0D088984203D1012901D1FFF79EFFB3
:1092500010BDC0462C68FF1FF0B5264E95B08700A4
:109260000B93BB590500099112200A92002B31D0B3
:10927000D888FFF7A5FB04001420002C2AD0280072
:1092800010A9FFF7B1FFBB591E781D6A002E23D02D
:109290000895FDF7EFFA07000020FDF7F1FA0790B7
:1092A000A379E61D069310AD0CA9089800F0E2FA28
:1092B0000EA9280000F0D7FA0B9B0A990493069B8D
:1092C00009980293079B0396019300970EAB0CAA93
:1092D000FFF77CFE15B0F0BDFDF7CCFA069030002C
:1092E000FDF7CEFAE31DA779079310AB06000893AC
:1092F000DAE7C0462C68FF1F30B50C4C85002A59B0
:10930000030085B00120002A0ED018006946FFF73F
:109310006BFF2B591A78D888054B002A00D1054BD2
:109320006A46072100F0D9FB05B030BD2C68FF1F4D
:10933000679800117598001130B5094C85002959BE
:1093400085B010226846253102F072FC2A5911219D
:10935000044BD0886A4600F0C0FB05B030BDC04663
:109360002C68FF1F1199001130B5094C850029594F
:1093700085B010226846353102F05AFC2A59112175
:10938000044BD0886A4600F0A8FB05B030BDC0464B
:109390002C68FF1F4F990011F7B54D4F8600102024
:1093A000F4590D0002F024FAF3592062186A1322CE
:1093B00000286CD0033A29009C6802F039FCF3596C
:1093C0001A780192002A58D11E6A227D317B944678
:1093D00051400122019F114201D167461740217D72
:1093E000914339432175377B4F40BC466046002787
:1093F000800701D44F081740012102208F40227DB1
:1094000082433A432275377B5740BC46604600276B
:10941000400701D497080F400420227DBF008243FB
:109420003A432275627D002794466046727B424033
:109430000A4201D167460F400121627D8A433A43C7
:109440006275777B5740BC4660460027800701D491
:1094500057080F400220627D7F00824317436775E3
:10946000767B00227E40760701D4BA080A400426A3
:10947000617D9200B1430A4362756A78002A08D080
:109480006278002A05D005220533DA770022100021
:10949000FEBD04222979114205D1A17C114202D1DD
:1094A0000533033AF1E7019A21782C78002A02D19A
:1094B0000A002100140018220429E8D8042CE6D858
:1094C00005206043034A05331218525CDDE7C046AD
:1094D0002C68FF1FECBF001110B50A001121024BD0
:1094E00000F0FBFA10BDC046AB9900110B0030B57F
:1094F00087B001AD2B806B4604001100981D082237
:1095000002F096FB2A000B212000024B00F0E5FA46
:1095100007B030BDD399001110B50A001121024BDC
:1095200000F0DBFA10BDC046279A001113B50B00FE
:1095300011006A4613706B4604000622581C02F0A4
:1095400077FB6A4608212000014B00F0C6FA13BDE4
:10955000479A001110B50A001121024B00F0BDFA24
:1095600010BDC046979A00117FB505000B4BAA00AD
:10957000D4580800002C0FD0666F237FE288217832
:109580000396266F0296E66E0196A46E0094FDF790
:1095900009FC2800FFF7FAFD7FBDC0462C68FF1FBD
:1095A00010B51721FFF7E0FF10BD000070B50A00ED
:1095B0000D00064B0221040000F08FFA0600297806
:1095C0002000FFF7D1FF300070BDC0467799001131
:1095D00070B586B000236A461370836804001D7856
:1095E000681E0A2859D801A902F0A2FA06063337E4
:1095F0003B3F43474B4F5300180000F042F906230E
:1096000012284BD000281BD16088FFF7D9F9082316
:10961000002813D04279002A47D1264B1A78072315
:1096200012070BD5244B1A680723002A06D01668A8
:10963000002E03D0290001AAB04703006A46137028
:109640006B461B786088002B2AD1FFF767FC06B0B9
:1096500070BD180000F06CF9D4E7180000F087F92D
:10966000D0E7180000F093F9CCE7180000F0ADF94E
:10967000C8E7180000F0C3F9C4E7180000F0F6F9D5
:10968000C0E7180000F0F6F9BCE7180000F013FA84
:10969000B8E7180000F013FAB4E707236A4613701E
:1096A00069466088FFF782FFD1E70523012AC5D10B
:1096B000024BB8E7B966FF1F2468FF1F2868FF1F29
:1096C000F8B52C4F8600F35904000D00002B40D054
:1096D000DA8882423DD15A78062A33D11A78002A94
:1096E0002ED0012099681A6A097D014206D0157BA7
:1096F000054203D007225A700120F8BD0220014222
:1097000004D0157B054201D00922F4E70420014270
:1097100004D0127B024201D00B22ECE7164B1B68EF
:10972000002BE9D05B68002BE6D020009847BB599E
:1097300000215B78122BDFD12000FFF715FFDBE75C
:109740000E4BECE7112A04D1002900D03225290064
:10975000F2E7002D08D12000FFF732F9002803D0EE
:10976000102302791343037121002800FDF798FAB2
:10977000C2E7C0462C68FF1F2468FF1F2868FF1F30
:1097800070B50E4E8500AB590400002B13D01B782A
:10979000002B11D10A4B1B68002B04D05B68002BF7
:1097A00001D02000984773595B78122B03D1002118
:1097B0002000FFF7D9FE70BD024BECE72C68FF1FBD
:1097C0002868FF1F2468FF1F094B8000C358102022
:1097D000002B0CD01A6A002A09D09B68002B06D0F7
:1097E000127A1B7E101C9A4200D9181CC0B2704716
:1097F0002C68FF1F70B503000D0014000220002A22
:1098000030D000292ED013700B78081D53704B7880
:109810009370FFF7A7FCE070012002212B7A2371DF
:109820006B7B034063716A7B0A40134304226371BC
:109830006E7B1640334363716E7BF608F60033434C
:1098400063712B7B0340A371287B014000200B43F5
:10985000A371297B0A401343A3712A7BD208D2004B
:109860001343A37170BD10B50A0001000120FFF77A
:10987000C1FF10BD10B50A0001000220FFF7BAFFBA
:1098800010BD70B506000C000220002E30D000295B
:109890002ED07378201D0B70B3784B70F178FFF7E2
:1098A0006DFC01223579257271794B100800134047
:1098B000934010400343881010408000C9080343C0
:1098C000C9000B436373B1794B10080013409340F8
:1098D00010400343881002409200C9081343C90096
:1098E0000B4321202373FCF773FE854201D2122023
:1098F00070BD2220257AFCF76BFE8542F7D82378CD
:109900001820042BF4D86378012BF1D80020EFE75E
:10991000030010B50220002909D0002B07D0032234
:10992000481C0A7019000D3202F082F9002010BDA7
:1099300003000222080010B5002B06D0002904D035
:109940000E32591C02F074F90022100010BD030001
:1099500010B50220002909D0002B07D00422481C92
:109960000A7019000C3202F063F9002010BD10B526
:10997000FFF7DEFF10BD03000220002906D0002BF8
:1099800004D0052200200A701B784B70704703003A
:109990000220002B08D0002906D05B7800200B7035
:1099A000013B082B00D918307047030010B5022086
:1099B000002909D0002B07D00622481C0A70190084
:1099C0000A3202F035F9002010BD10B5FFF7B0FFE4
:1099D00010BD02000B00022010B500290ED0002A95
:1099E0000CD007211970118859701188090A9970D3
:1099F00011180822D81C02F01BF9002010BD03002A
:109A00000A00022010B5002B0CD000290AD099784A
:109A10005878090201431180901CD91C082202F0D9
:109A200007F9002010BD030010B50220002909D05D
:109A3000002B07D00822481C0A701900921802F067
:109A4000F7F8002010BD02000B00022010B500291D
:109A50000BD0002A09D009211970117818185970F3
:109A6000511C062202F0E4F8002010BD10B5FFF7EB
:109A70005FFF10BD02000B00022010B5002A09D0C4
:109A8000002907D05178197011180622581C02F0CD
:109A9000CFF8002010BD030010B50220002909D026
:109AA000002B07D00A22481C0A701900063202F067
:109AB000BFF8002010BD10B5FFF73AFF10BD02003F
:109AC0000B00022010B5002A06D0002904D018008F
:109AD0005178FFF753FB002010BDF0B585B017009B
:109AE0001E006A4606230500080091819380FEF758
:109AF000C0FC1324011E02900CD03800B047041E95
:109B000005D1280001A9FEF76FFA041E02D00298C1
:109B100001F00EFE2800FFF701FA200005B0F0BDAD
:109B2000F0B504008BB0019115000021102202A8AD
:109B300002F066F8334EA700B85900283CD0C3881D
:109B4000A34239D10378002B36D14278062A18D1A6
:109B500002000100553235310C3006ABFFF7A9FA8F
:109B6000002829D12000FFF72FFE020006A902A835
:109B700002F05EF8200002A901F01AFE01200BB0ED
:109B8000F0BD816E002917D00B8A112A28D19D4281
:109B90000ED101981231093A01F0E2FF012807D1F4
:109BA000BB5920009D6EFFF70FFE29000200DEE783
:109BB00032212000FFF7D8FC2000FEF701FF061E2F
:109BC0001BD0416A002918D00B8AAB4215D108225C
:109BD0000198123101F0C4FF01280ED1716A0AE028
:109BE0009D42E9D108220198123101F0B9FF012804
:109BF000E2D1BB59996E8A7EB9E7200001F070FD71
:109C0000BCE7C0462C68FF1FF0B56B4D87007E593E
:109C100085B0337802900393002B00D087E0B368BF
:109C2000346A01937078062817D101221B7D1342F4
:109C300002D0217B114218D10222134202D0217B93
:109C4000114251D10422134203D0237B134200D08E
:109C50008BE0019B5A7DEB5991E007380428F8D836
:109C600001F066FF032E42678300B36E002B03D121
:109C70001C2001F0BDFDB066EB599C6E002C1CD081
:109C800010220021200001F0BBFF0298FFF79CFD8D
:109C900001002000FFF72DFA01F0A2FD2082200034
:109CA00008211230FFF725FA0298FFF78DFDA07604
:109CB000EB592100D888FFF70FFC0822EB591CE074
:109CC000B36E002B05D01A00198AF0881232FFF704
:109CD0000DFC0222019B197DEB5911423DD0207BE6
:109CE00010423AD0073208E0F488FCF7DBFD0100AF
:109CF0002000FFF711FC0A22EB595A70029B9C00CE
:109D00002A595378073B042B11D8D088FEF758FE08
:109D100000284ED0C3895A08D2182849029B0298BD
:109D2000CB542B5941180433254801F0C1FF05B02D
:109D3000F0BDFCF79FFD03000120834201D100200C
:109D40000393EB59DE88FCF79BFD0399020030007A
:109D5000FFF7ECFB019AEB59117D042211420CD064
:109D6000217B114209D00B22C7E7F688FCF73CFDA6
:109D700001003000FFF7EEFB6BE7019A527D0121F5
:109D80000A4204D0607B084201D00C22B5E70221D0
:109D90000A4204D0607B084201D00E22ADE70421C4
:109DA0000A4204D0627B0A4201D01022A5E71222A7
:109DB000A3E7FA225200B0E72C68FF1F3068FF1FAC
:109DC0007FA1001110B5064B1A780423100018402B
:109DD0001A4200D00348FFF727FA002010BDC04602
:109DE000B966FF1F3C45FF1F70B50400FFF7D4FAAA
:109DF000051E43D12000FFF77FFA234EA400A0598F
:109E00008268937CDB0708D50321036A1B790B402A
:109E1000012B02D1017F0B430377431DD97F8B1E9A
:109E2000022B0DD8022900D00121C088FCF790FF39
:109E3000042133591A7F59700A431A77280070BDDC
:109E400001290CD102231022437000210C3001F0B3
:109E5000D7FE305910213530FFF74BF9EEE70529D1
:109E6000ECD10223D118437010220C3001F0E0FE37
:109E700004233259117F0B431377EAE7082518288A
:109E8000DCD1053DDAE7C0462C68FF1FF0B58BB08A
:109E9000059143887E4F9E00F45915000493002CD1
:109EA00015D1012902D000200BB0F0BD101D57784C
:109EB0001678FFF757F9EB68320002932B7A049972
:109EC000019300903B002000FCF70CFFEBE7E388D8
:109ED000049A934201D00820E6E72378012B00D1B1
:109EE000D4E0059B581E092800D9CFE001F020FEE0
:109EF00005CE0A29CC506C859AB229000498FFF748
:109F000073FFD1E7200029001022453001F090FEB8
:109F1000B9594B78042B02D1013B4B70C3E70B00BE
:109F20000A00253335320C310498FFF795F904986F
:109F3000FFF702FA0522431E9841BB59C0005A7030
:109F4000B2E7200029001022553001F071FE049B79
:109F50004F4C9D00295904980A0006AB55320C312C
:109F6000FFF77AF929591022453106A801F0F8FDCA
:109F7000012808D10498FFF7F7F90590002804D1CB
:109F800006222B595A7005988EE708230593FAE7A5
:109F900063780C2B7AD1E36E002B03D11C2001F0E7
:109FA00027FCE066BB59D86E00286FD0102229002C
:109FB00001F03EFEBB590498DC6EFFF705FC0D2254
:109FC000A076BB595A706EE7E06E00285ED06378C9
:109FD0000D2B5BD12B8808220382A91C123001F0C3
:109FE00027FEBB599A68517D0222114226D0186A79
:109FF000407B104222D00C32E4E763780E2B45D12F
:10A00000236F002B03D1162001F0F2FB2067BB5910
:10A01000186F002803D01022290001F009FE0F223A
:10A02000BB59CFE763780F2B30D1206F0622691C14
:10A03000103001F0FDFDBB599A68517D0422114298
:10A0400003D0196A497B1142D5D100210498FFF74A
:10A050008BFA28E7636F002B0DD0BB59586F00288F
:10A06000F3D01022290001F0E3FD0122BB59524236
:10A070005B6F1A61E9E7142001F0BAFBBB59606716
:10A080005B6F002BE9D126E72978DFE707200BE794
:10A090002C68FF1F10B5064C207001F0D9FC06217A
:10A0A0002078FDF791FF0348FEF778FC10BDC0460D
:10A0B0003F68FF1F3592001100200BB270B50D00F4
:10A0C000834216DA264B187801F06AFD041E0DD083
:10A0D0000378922B0ED0A02B37D0224B1878FF2874
:10A0E0003AD0210001F03CFB002835D1802000024D
:10A0F000684070BD43780E2B0BD03E2BEDD183789A
:10A10000052B12D0082BE8D181798088FFF7D8FA87
:10A1100008E0154B82889A42DFD183681878591C71
:10A12000FEF7C0FE002817D1D7E7104B1B785B075E
:10A1300012D50F4B1B68002B0ED09B68002B0BD049
:10A14000C289811D80889847ECE7FFF741FAA06833
:10A15000002801D001F0ECFA200001F0F9FAC5E77F
:10A160003F68FF1F3545FF1F18200000B966FF1F1D
:10A170002868FF1F10B50078FFF712FA10BD10B560
:10A180000078FFF7FDFA10BD0C234343084A10B5D1
:10A190009B185A68002A03D0012901D1904710BDAD
:10A1A0009B68002BFBD00029F9D19847F7E7C04600
:10A1B0005C68FF1F01238340094A10B5946B1C4360
:10A1C0009463506B98435063D46B200098430129EB
:10A1D00001D120001843D063116B0B43136310BDF2
:10A1E00000800040F0B500240127154B85B0DA6BE4
:10A1F000144E03921A6C0192DA64019BE3403B42D5
:10A2000017D0039DE5403D400295E5B20299280034
:10A21000FFF7BAFF316A736A002908D03900002BB2
:10A2200001D0029979402800FFF7C4FF01E0002B1C
:10A23000F9D101340C36172CDFD105B0F0BDC04682
:10A24000008000404068FF1F064B01215A68C24051
:10A250000A4204D01B68C3401800084070471B6DB9
:10A26000F9E7C046008000400122064B82400029E9
:10A2700003D0D9680A43DA607047D9689143D9603E
:10A28000FAE7C0460038004030B5032444430F4B82
:10A29000E25C1B199C785D7801232D1B0135AB40D6
:10A2A000013BA340A140DB430C00122807D808491A
:10A2B00092005218116819402143116030BD054ABF
:10A2C00011680B4023431360F8E7C04633C0001108
:10A2D00008F0004014F00040C21F70B5D4B206234D
:10A2E000092C0BD80125084C9540002908D00021E5
:10A2F000FFF7CAFF23682B4323600023180070BDBB
:10A300002368AB43F8E7C04600380040214BF0B566
:10A310001B185B78022B21D1032444431E4A1F4E95
:10A32000A35C12199478012215008540B76B013C9B
:10A33000E4B23D43A240B563194C122815D89B00E6
:10A3400000290CD117495B1899680A439A600123C8
:10A35000205C154A834011680B431360F0BD11491E
:10A360005B18996891439960F1E70E4B00290DD174
:10A3700059690A435A61225C1328E8D00123203A24
:10A3800093400A49086803430B60E7E75969914322
:10A390005961F0E74068FF1F33C0001100800040A2
:10A3A00078C0001100F00040A0F00040A4F0004090
:10A3B000F8B500241B4E1C4D1C4B1B5D012B1FD1FF
:10A3C000194A9269E2401A420BD00122B2569340D8
:10A3D0002200143AD2B2022A09D815494A69134315
:10A3E0004B61013402360C35172CE5D1F8BD002243
:10A3F000B2560F499200521891680B439360F0E7F0
:10A40000022BEED1E7B23800FFF71EFF01235840C0
:10A41000C1B23800FFF77AFF3800FFF715FF687701
:10A42000DFE7C04605C000114068FF1F4168FF1FFD
:10A4300000F00040012202388240054B002903D081
:10A4400059690A435A617047596991435961FAE75A
:10A4500000380040F8B50E0001210F008740114A76
:10A460000400D368FD43BB43D360831E8B4201D8F5
:10A47000FFF7E0FF00212000FFF72EFF0A4A0B4BF9
:10A480005168012E05D139431B1951605E700020BF
:10A49000F8BD2940516002221C1962709A6915406A
:10A4A0009D61F4E700380040008000404068FF1FD5
:10A4B000012210B58240074B002906D019680A43D3
:10A4C0001A600121FFF7C6FF10BD1968914319609A
:10A4D000F7E7C046008000400C2370B500254343D9
:10A4E0000A4A29009B181D70094B04001B185D7057
:10A4F000FFF7B0FF0123A340064928000A681A436A
:10A500000A6005490A689A430A6070BD5C68FF1FCB
:10A510004068FF1F348000403080004070B5040068
:10A520000E00FF2813D003250540FFF7D5FF084A8A
:10A53000A3089B009B183F22ED00AA40AE4019687B
:10A5400020009143314319600121FFF78DFE70BD5A
:10A5500018380040F8B50C244443134B0500E418A8
:10A560006368002B03D1A3681220002B1AD00222AB
:10A5700001270E4B00215B195A7028002770FFF746
:10A5800069FF63681E1E08D0A3683E00002B04D03C
:10A590002800FFF759FE4640F6B228003100FFF7C9
:10A5A00009FE0020F8BDC0465C68FF1F4068FF1F21
:10A5B000F7B5C420FF222B4B80001958002491438B
:10A5C0003F3A0A431A508022274F5202274E1A6000
:10A5D000274B1D5D002D21D0A31E012B03D8012187
:10A5E000E0B2FFF727FF012D18D11F4B9B69E34015
:10A5F0002B4213D0E3B218000193FFF725FE0100B0
:10A600000198FFF755FFE3B2143B022B1DD801213F
:10A610007156184A8D405369AB4353613B7F002B01
:10A620000DD0E5B22800FFF795FF2800FFF70CFEDC
:10A630007B7F0100834202D02800FFF7A5FD013493
:10A640000C370236172CC3D1F7BD012100237156F8
:10A65000F3568D40074A9B009B189A68AA439A605C
:10A66000DCE7C04600E100E04068FF1F05C00011C4
:10A670004168FF1F00F0004010B501210400FFF702
:10A68000E9FE0123044A002011194B70A34091698F
:10A690000B43936110BDC0464068FF1F70B50E00AC
:10A6A00015000400FFF718FF0C236343094A20003C
:10A6B0009B189D605E60FFF74DFFF021064B074A37
:10A6C0008900051E5A5002D02000FFF705FF280020
:10A6D00070BDC0465C68FF1F0000FF1FE5A10011B0
:10A6E00070B5134D07202C78002C1FD19822210023
:10A6F0005200280001F08CFA0123C420FF222B70A5
:10A700000C4B80001C635C630B4B1C605C600B4B50
:10A71000195891433F3A0A431A50802252021A6054
:10A720000D20074A074901F04BFA200070BDC046D2
:10A730004068FF1F00800040A0F0004000E100E002
:10A74000B1A50011B1A30011030010B50620072B1D
:10A7500009D8054A137001F02BFAD7210020034BCA
:10A76000034A89005A5010BD6445FF1F0000FF1FB7
:10A77000151BFF1F70B51D0002240C2910D8094AB3
:10A78000CA40D2070CD5FBF72FFF041E08D1059A4B
:10A7900004992800FBF744FFFCF7B2FDFFF712FB1A
:10A7A000200070BD1210000030B50D7802232C007F
:10A7B0009C43184201D02B431C0008252300AB43C7
:10A7C000284201D02B00234320241D00A543204212
:10A7D00001D01C4325002A230D70184204D01178A3
:10A7E0001E3B0B43137030BD0028FCD10C211378A5
:10A7F0008B43F7E7F8B51D0006AB1B88140007AACA
:10A800000E000B201778002B27D10A78022A49D195
:10A810004A68507811780002244A084380180428B6
:10A8200040D801F085F903121D1B2300F06801F0E8
:10A83000B7F8021CC0B2B84200D93A1CD2B220000C
:10A84000F1682A8001F0F4F906E00222F3681B881F
:10A850002A8023701B0A63700020F8BD0622EEE7F1
:10A8600001232B80F3681B782370F5E7F368002B36
:10A8700016D008222A801A8822701A88120A62705A
:10A880005A88A2705A88120AE2709A8822719A88AD
:10A89000120A6271DA88A271DB881B0AE371DBE7B6
:10A8A0002B80D9E701202B80D7E7C04600D6FFFFD9
:10A8B000F7B516000A781D0008AB1F880C000123AD
:10A8C000022A18D14A685078117800022B4A0843AE
:10A8D000801803280FD801F02BF902254439E068CD
:10A8E00001F05EF8C0B20723B84204D37B1901938C
:10A8F000152B02DD0D231800FEBDE0682A00310093
:10A90000C01901F095F96B4600209B88E268D0548D
:10A910001B4B1B68834203D01B68834200D09847BF
:10A920000023E8E70B23002FE5D1022DE2D1737855
:10A9300032781B021343E2681380114B1B68002B13
:10A94000EED01B68002BEBD00120E8E70B23002F93
:10A95000D1D1062DCED12A003100E06801F068F98E
:10A96000DEE70B23002FC6D1012DC3D1327875331A
:10A97000012AC0D8E3681A70D2E7C04600D6FFFFAC
:10A980004C6AFF1F70B50C001500072837D801F07E
:10A99000CFF8041436361B36242E182015290BD870
:10A9A000184E16220021300001F02AF92200290059
:10A9B000300001F03DF9002070BD18200229FBD1C4
:10A9C0001288114B1A80F6E718200829F4D10A00E2
:10A9D0000E48290001F07CF8EDE718200129EBD1A1
:10A9E0000B4B10780B49DA69FFF7DEFEE3E718201E
:10A9F0000129E1D1064B10780749DA6BF4E7022010
:10AA0000DAE7C046346AFF1FE245FF1FD845FF1F43
:10AA10006845FF1F9045FF1FB045FF1F030010B59D
:10AA20000020DB0704D50721024A034800F08CF818
:10AA300010BDC04690C000116845FF1F054A0300C5
:10AA40001068002803D082889A4201D1806870473C
:10AA50000068F6E7506CFF1F0A88030008009A425E
:10AA600004D08A8804309A4200D000207047000049
:10AA7000F8B5F82200230D4F0D4E796805004243CA
:10AA80003370994200D07B600A4C0021200001F015
:10AA9000B7F800231A007C60AB4202D1002033706B
:10AAA000F8BD01332280DBB2F834F5E7506DFF1FAB
:10AAB0004C6DFF1F546CFF1F73B56B460190060071
:10AAC000684615001980FCF74DFF041E11D1002DBA
:10AAD0000FD07689002E11D00C2000F089FE0028BE
:10AAE0000ED0084A0460136886808560002B02D16E
:10AAF0001060200076BD1A001B68F7E70224F8E713
:10AB00001324F6E7506CFF1F012100220A4B10B5F9
:10AB100049420A4C198099809A719A70084B2070AA
:10AB2000012019805A60FFF7A3FF2078FCF778FF17
:10AB30000448FDF733FF10BD546AFF1F586DFF1F17
:10AB4000506DFF1FF5AB0011022310B5002802D095
:10AB5000FFF7B2FF0300180010BD0000030010B59E
:10AB60000020DB0704D50421024A0348FFF7A4FFB5
:10AB700010BDC046A4C00011E845FF1FF0B50E2669
:10AB800087B003930CAB1F8802ABF61805000800D2
:10AB900031000292FDF768F804000120002C0FD06C
:10ABA0003088FFF74BFF03000E20002B08D05E68B3
:10ABB000002E05D021002800039B029A0097B04781
:10ABC00007B0F0BD0A4B10B5984207D1012200230F
:10ABD00052420A808B708A808B7110BDFFF73CFF58
:10ABE0000028FAD001235B42038000238370F4E73E
:10ABF000FFFF0000F8B5050001290AD1134E00241B
:10AC00003388F827AB4219D028001149FFF7DAFF43
:10AC100006E0022904D10139FDF73EFF0028EDD0FE
:10AC2000F8BD3B0063437268D018D35A002B09D09B
:10AC30003A00002100F0E4FF0134E4B2054B1B7838
:10AC4000A342EED801235B423380DDE7506DFF1F46
:10AC5000546AFF1F4C6DFF1F10B5FFF7FDFE030088
:10AC60000020834200D0987810BD0000F0B589B074
:10AC70001C000EAB80CB03901E8810AB1B78049297
:10AC800002930B7A0D00DB0616D42B780593022B6A
:10AC900024D00498FFF7D2FE002812D003689C4607
:10ACA000002B0ED0029B2200019329003B0064463A
:10ACB00003980096A04705E00498FFF7BFFE002820
:10ACC00002D10E2009B0F0BD8368002BF9D00A2212
:10ACD0002900039898470028D7D0F3E76B68587885
:10ACE0001A786B4B000210439842D2D8043B98422A
:10ACF00010D2684B984242D015D8674BC018012833
:10AD0000C7D80B20002EDDD1EB681A7859683A803D
:10AD1000200028E0614BC018032800D979E000F03A
:10AD200007FF846A789E5E4B9842B2D10B20002EBA
:10AD3000C8D101233B80EB6831001B782370688900
:10AD4000013080B2FCF790FF3A88031E0ED00178E4
:10AD500002328A183A80428962704289120AA270CD
:10AD600059680278E01C00F063FF06E004323A8084
:10AD700031000422601C00F043FF0020A2E70B20FA
:10AD8000002E9FD1EB6807A91E8804233B80330A5D
:10AD9000300026706370FCF767FF051E28D004ABF7
:10ADA0009A890E2304A95B183E49C668FCF7D0FFB8
:10ADB00000280BD12B783C486A680599FBF786FB85
:10ADC000002803D1012304AA5B42D3813278022AEE
:10ADD00006D17168201D00F02BFF3B8802333B80B9
:10ADE0000E2304AA9B181B88A3701B0AE370C4E7F8
:10ADF00004ABDE81F4E70B20002E00D062E7E968A7
:10AE00000398FFF729FF02233B802070000A60703F
:10AE1000B3E70B20002E00D054E70222EB681B881A
:10AE20003A8023701B0A6370A7E7E86800F0B8FD5A
:10AE3000C2B203000720B24200D243E70DD002990C
:10AE4000DBB27118994202DB921BD3B20293029BD0
:10AE5000E9681A003B8089195AE70023F6E70B20BE
:10AE6000002E00D02EE70722EB683A801A78227075
:10AE70005A7862705A88A2705A88120AE2701A7957
:10AE80002271DA886271DB881B0AA37175E7C046FC
:10AE9000042900000228000000D8FFFFFFD6FFFFB2
:10AEA00003280000FFFF0000D4BF0011F0B58DB0F3
:10AEB0006B460020089120229B5E83423DDAA64B20
:10AEC000187800F06DFE071E32D00378B02B2CD11D
:10AED0000079023816281FD800F0D2FC17001E0097
:10AEE0001E001E0031001E0096001E001D011E00E7
:10AEF00052011E0073011E00CD011E0050021E00F3
:10AF00001E001E008E021E00E302944B94491B8813
:10AF100078880B80FBF71AF83800FCF79BFF914B01
:10AF20001B68002B01D038009847380000F010FC57
:10AF30008020089B0002434018000DB0F0BDF622AF
:10AF40000021874800F05CFE0BAA3B7B7989388999
:10AF500000923A000D32FCF79FFD0400804B1B78F5
:10AF6000002C3FD146E0804B788805937F4B410011
:10AF7000CB5A0BAE073BDBB232880293002301931E
:10AF80007B4B210006930093059BFFF76FFE744DEA
:10AF9000002810D1069B3A8A1B889A420BD13800B0
:10AFA0000599123000F0DCFD002804D02B7862896E
:10AFB0009B00EB185A80162306A81B183288200025
:10AFC0007989FCF7C5FE2B7804009A00AA185188ED
:10AFD0000029C3D00133DBB22B70002807D006A9AB
:10AFE000C98A9180634A12889A42BCD802E0012142
:10AFF00049429180002B04D059497888FAF7DAFF4A
:10B000008AE73E890A2479E000253E89574B06935A
:10B010007B88069A5B009B5A033B9D4202DB002D16
:10B02000F0D05BE0162206A812183B7B79890092CB
:10B030003A0030000D32FCF72FFD0590002858D063
:10B040004689017A7888FCF7F1FC041E44D1464B0E
:10B0500078880793069B4100C95A454B0439C9B209
:10B0600006AAD28A06930291019400930599079B40
:10B07000FFF7FCFD041E2FD1069B39491A88931C4B
:10B08000002D26D14B807988384B4900CB5A511975
:10B09000033B8B4220DD059B31485B8941190B71D5
:10B0A000A91C0135C9B2EDB2059145191B0A2B71D6
:10B0B000059B2D490433181800F0BAFD2C4B059A56
:10B0C0001B88D318DDB22C4B9E4205D00136B6B298
:10B0D0009CE749889942D6D0002D0CD0204C2800FE
:10B0E000618800F0BDFC207021007888FAF772FFBB
:10B0F00012E7059CF0E7002C00D183E77B78142B46
:10B1000000D109E716493B794E800B700C717888A5
:10B11000FAF712FF00E7162406ABE418210038897D
:10B12000FCF7A2FD011E00D1B7E1788822880F4C00
:10B1300045002C5B0A4D013CE4B2029400240F4B05
:10B1400001940095FFF792FD041E00D014E1290040
:10B150007888FAF74FFFDFE6586DFF1FD444FF1FD2
:10B160005C6AFF1F506AFF1F566BFF1F8C66FF1F34
:10B170004C6CFF1FD244FF1FFFFF00005E6AFF1FE1
:10B18000162406ABE41821003889FCF76DFD011E7A
:10B1900000D182E178882288AE4C45002C5BAE4D10
:10B1A000013CE4B202947C89AC4B01940095FFF71A
:10B1B0005DFD041E00D0DFE029007888FAF724FF47
:10B1C000AAE60025A44B1D803B00FE331B78A24A53
:10B1D00078880792AB4208D99E4B1288069306994D
:10B1E00043005B5A013B9A4203DB0799FAF716FFCB
:10B1F00092E616246B00FB18059306ABE418059B3A
:10B2000021001889FCF730FD011E03D1059B0124A4
:10B210001E8973E77888924B2288069C0993430025
:10B220001B5B904E013BDBB202930023009601931F
:10B23000099BFFF71BFD041E02D0059B1E895DE7DD
:10B240007B88069A5B009B5A079A108832881218EE
:10B25000934202DC1B1A013B33807F4C0230328860
:10B260000999001900F0E4FC2388328801359B1805
:10B270002380EDB2A8E70BAA3B7B7989388900923D
:10B280003A000D32FCF708FC00250590059B002BC9
:10B2900004D10A24002D00D16EE060E0059B78887F
:10B2A000197AFCF7C3FB0100041E63D1694C6C4B97
:10B2B000788806940993069B4400E45A694B063C3F
:10B2C000E4B20BAE32880793029401910093059982
:10B2D000099BFFF7CBFC041E4CD1079B5E491B88E2
:10B2E0001A1D002D30D14A80059B5B4C5A89631989
:10B2F0001A716B1C9BB2E318120A1A71162306A866
:10B3000032881B1879890598FCF722FDFF21AA1CB9
:10B310002E1D03350B00059092B2B6B2ADB20028D7
:10B3200003D006ABDB8AD9B21B0AA21865191171CA
:10B330002B714C4D301D2A884949201800F078FCAB
:10B340002B88F618B5B2A1E74988914207D17A88CF
:10B3500006995200525AEB18053A9A42C4DC3E4C08
:10B360002800618800F00CFB207021007888FAF733
:10B370005FFED1E5002DF2D13E89BFE6162606AB71
:10B38000F61831003889FCF76FFC3D000400FF35EA
:10B3900000282DD0037A9B060CD400227B893989A2
:10B3A000788800923A000C32FFF7E8FB041E10D0B8
:10B3B0003E8915E03088FFF741FB00281AD08368EA
:10B3C000002B17D02100122278889847041EE4D061
:10B3D000EEE7AB78002B02D17888FAF739FE002629
:10B3E000AB78002B00D097E5002C00D194E585E6E2
:10B3F0000124DDE70E24DBE7162506ABED18290056
:10B400003889FCF731FC041E47D0037A9B0611D41F
:10B41000154A7B881188994203D01448814207D18C
:10B420001380134BF8261D780023D9B2A94221D3EB
:10B430000924A1E72888FFF701FB00282FD08368A3
:10B44000002B2CD02100122278889847041EDFD0D0
:10B4500092E7C0468C66FF1F5C6AFF1F5E6AFF1F93
:10B46000566BFF1F4C6CFF1F506DFF1FFFFF00004E
:10B470004C6DFF1F31005943546801336018615A05
:10B480000029D2D13C0008342100F82200F0D0FB82
:10B4900021007888FAF7E4FD3EE501246CE70E24EC
:10B4A0006AE71D4B1A887B889A4231D07888FAF770
:10B4B000E1FD31E5F823059851684343CD18C95A99
:10B4C00000291FD03B7A012B0BD16C88AB88788880
:10B4D000AA1D0094FFF752FB041E02D000233B720A
:10B4E0002E88F8220021280000F08AFB00232B8000
:10B4F000059B0133DBB20593084B05991B78064A7F
:10B500008B42D7D801235B421380002CCED0F5E5C7
:10B51000002634000596EFE7506DFF1F4C6DFF1FAE
:10B5200070B504000E001500FFF796FA031E08D14F
:10B5300031000548FFF790FA03001120002B02D0DC
:10B540001C8000209D7070BDFFFF0000F8B50B4F00
:10B5500006003B780D001400FF2B0ED00A2000F0EF
:10B5600007FA011E09D0B12303800023468003712E
:10B57000C5800481387800F0F3F8F8BD2946FF1F34
:10B58000F7B50F0008A90600088809A90B24098847
:10B59000002821D10234022B1ED1557813782D02B8
:10B5A0001D432B008B4301937334002B14D1FB6894
:10B5B000300019000093FFF74FFB019C85420BD030
:10B5C0002A0030000099FFF7ABFF041E04D12A00C7
:10B5D00030007989FFF7BAFF2000FEBDF0B50E7884
:10B5E00085B003900AA805880120022E0DD14C6871
:10B5F0002778647824023C43054FBC4205D1039868
:10B60000DBB201960095FFF7BBFF05B0F0BDC04669
:10B610000229000010B504000C4800F069F80C483D
:10B62000A16B00F065F80B48E16B00F061F80A4887
:10B63000216C00F05DF8094B0948196800F058F8D2
:10B64000084B1B68002B00D09847FEE786BE001110
:10B650009CBE0011ABBE0011BABE001104ED00E0AB
:10B66000C9BE00115C6DFF1F002307B501A801933F
:10B67000FFF7D0FF044A0548002110B5121A00F068
:10B68000BFFAF8F797F9FEE7606DFF1F2C46FF1F22
:10B6900001B40248844601BC604700BF7132FF1FFD
:10B6A00001B40248844601BC604700BFED4A010076
:10B6B00001B40248844601BC604700BF090E000087
:10B6C00001B40248844601BC604700BFC5210000A8
:10B6D00001B40248844601BC604700BFC53F00007A
:10B6E00001B40248844601BC604700BF091B00004A
:10B6F00001B40248844601BC604700BFE53A01003E
:10B7000001B40248844601BC604700BF156B0100CC
:10B7100001B40248844601BC604700BF21240000F8
:10B7200001B40248844601BC604700BFE13CFF1FF2
:10B7300001B40248844601BC604700BFD9490100FA
:10B7400001B40248844601BC604700BFC537FF1FF3
:10B7500001B40248844601BC604700BF434D01006C
:10B7600001B40248844601BC604700BF594F010044
:10B7700001B40248844601BC604700BF6571010006
:10B7800001B40248844601BC604700BFC94A0100B9
:10B7900001B40248844601BC604700BF8B520100DF
:10B7A00001B40248844601BC604700BF014C01005F
:10B7B00001B40248844601BC604700BF311B000051
:10B7C00001B40248844601BC604700BF55490100EE
:10B7D00001B40248844601BC604700BF1147010024
:10B7E00001B40248844601BC604700BF29510100F2
:10B7F00001B40248844601BC604700BF3D4B0100D4
:10B8000001B40248844601BC604700BF3D180000F7
:10B8100001B40248844601BC604700BF913AFF1F53
:10B8200001B40248844601BC604700BF75A900000E
:10B8300001B40248844601BC604700BFC51D00003A
:10B8400001B40248844601BC604700BF691F000084
:10B8500001B40248844601BC604700BF4551010065
:10B8600001B40248844601BC604700BF4939FF1F4C
:10B8700001B40248844601BC604700BF791800004B
:10B8800001B40248844601BC604700BF093DFF1F68
:10B8900001B40248844601BC604700BF513AFF1F13
:10B8A00001B40248844601BC604700BF851F000008
:10B8B00001B40248844601BC604700BF9538FF1FB1
:10B8C00001B40248844601BC604700BF6DBC000063
:10B8D00001B40248844601BC604700BFA137FF1F86
:10B8E00001B40248844601BC604700BFDD66010028
:10B8F00001B40248844601BC604700BF5D170000E8
:10B9000001B40248844601BC604700BF0124000026
:10B9100001B40248844601BC604700BF056A0000CC
:10B9200001B40248844601BC604700BFE53BFF1FED
:10B9300001B40248844601BC604700BFE92800000A
:10B9400001B40248844601BC604700BF5125000095
:10B9500001B40248844601BC604700BF5135FF1F57
:10B9600001B40248844601BC604700BFADAE000090
:10B9700001B40248844601BC604700BF1D4D010070
:10B9800001B40248844601BC604700BF090E0000B4
:10B9900001B40248844601BC604700BFEDA5000029
:10B9A00001B40248844601BC604700BFDD5201007B
:10B9B00001B40248844601BC604700BFA54F0100A6
:10B9C00001B40248844601BC604700BFB54C010089
:10B9D00001B40248844601BC604700BFE54800004E
:10B9E00001B40248844601BC604700BFB93BFF1F59
:10B9F00001B40248844601BC604700BFE530FF1F28
:10BA000001B40248844601BC604700BFB352010044
:10BA100001B40248844601BC604700BFB134FF1F37
:10BA200001B40248844601BC604700BF25260000DF
:10BA300001B40248844601BC604700BF5147010081
:10BA400001B40248844601BC604700BFC932FF1FF1
:10BA500001B40248844601BC604700BFC92600000B
:10BA600001B40248844601BC604700BF350E0000A7
:10BA700001B40248844601BC604700BF193AFF1F69
:10BA800001B40248844601BC604700BF350E000087
:10BA900001B40248844601BC604700BF0189000030
:10BAA00001B40248844601BC604700BF4550000015
:10BAB00001B40248844601BC604700BF7D18FF1FE7
:10BAC00001B40248844601BC604700BF0D5201002A
:10BAD00001B40248844601BC604700BF810E0000EB
:10BAE00001B40248844601BC604700BF8932FF1F91
:10BAF00001B40248844601BC604700BF9930FF1F73
:10BB000001B40248844601BC604700BF017F0000C9
:10BB100001B40248844601BC604700BFD1A50000C3
:10BB200001B40248844601BC604700BF355500009F
:10BB300001B40248844601BC604700BFF53CFF1FCA
:10BB400001B40248844601BC604700BF4136FF1F74
:10BB500001B40248844601BC604700BFD91B000005
:10BB600001B40248844601BC604700BFCD4C0100CF
:10BB700001B40248844601BC604700BF053AFF1F7C
:10BB800001B40248844601BC604700BF2146010061
:10BB900001B40248844601BC604700BFC95C010093
:10BBA00001B40248844601BC604700BFF54E010065
:10BBB00001B40248844601BC604700BF151BFF1F4B
:10BBC00001B40248844601BC604700BF1133FF1F27
:10BBD00001B40248844601BC604700BFE117000081
:10BBE00001B40248844601BC604700BFB14E00006A
:10BBF00001B40248844601BC604700BF55220000E2
:10BC000001B40248844601BC604700BF154D0100E5
:10BC100001B40248844601BC604700BFB70E000073
:10BC200001B40248844601BC604700BFD13AFF1FFF
:10BC300001B40248844601BC604700BFE94C0100E2
:10BC400001B40248844601BC604700BF055E0000A5
:10BC500001B40248844601BC604700BF3D3BFF1F62
:10BC600001B40248844601BC604700BFF30E0000E7
:10BC700001B40248844601BC604700BF9DA9000092
:10BC800001B40248844601BC604700BFC56D010095
:10BC900001B40248844601BC604700BFF94C010072
:10BCA00001B40248844601BC604700BF59520100FC
:10BCB00001B40248844601BC604700BFA9460100A8
:10BCC00001B40248844601BC604700BF1D4B01001F
:10BCD00001B40248844601BC604700BF8D120000D9
:10BCE00001B40248844601BC604700BF8552010090
:10BCF00001B40248844601BC604700BFF134FF1F15
:10BD000001B40248844601BC604700BF4D1F0000DB
:10BD100001B40248844601BC604700BF456B010086
:10BD200001B40248844601BC604700BFC9A90000B5
:10BD300001B40248844601BC604700BF291C0000D2
:10BD400001B40248844601BC604700BF5118FF1F80
:10BD500000020103020203030403050206020702B4
:10BD6000080209030A030B030C020D000E030F0364
:10BD7000100311031303140315001600913D001165
:10BD8000C53D0011000000000200000092BD00113E
:10BD9000192A0F180A000000F1590000FD240000C4
:10BDA00041460100A5800011B9A000110D750011D8
:10BDB000A97E0011B1530011ADAE00111950001150
:10BDC000893F0011B9400011000000001616000064
:10BDD00002000000DCBD0011F4FFF3FFD2FC000004
:10BDE000F941001100000000000000005475796165
:10BDF0000042312E3200303031340067697468758A
:10BE0000622E636F6D2F707676780054483035005F
:10BE10000200000024BE0011292A282A272A262AE7
:10BE2000252A242A0A180000E204000071020000FA
:10BE300078EC0000744000001027000060F0000063
:10BE400006640000204E0000000000000100000019
:10BE50001F501D00023CB40000011500120000003C
:10BE6000A10200003031323334353637383941429F
:10BE700043444546005048592B36325858504C558B
:10BE80005330353034005B48617264206661756CF4
:10BE9000742068616E646C65725D0A004C522020EB
:10BEA000203D203078253038780A0050432020206B
:10BEB0003D203078253038780A0050535220203DFC
:10BEC000203078253038780A0049435352203D20ED
:10BED0003078253038780A00B5570011095800111C
:10BEE0000000000002000000F0BE00116F2A6E2A60
:10BEF0001A18EAC8BC80F0FC60FFFFFFFFFFFFFFDD
:10BF0000FFFFF303B59747D6F613F7D777E6F0A709
:10BF1000F474000001A00000000000006410B71DD0
:10BF2000C8206E3BAC30D9269041DC76F4516B6B67
:10BF30005861B24D3C7105502083B8ED44930FF029
:10BF4000E8A3D6D68CB361CBB0C2649BD4D2D386DF
:10BF500078E20AA01CF2BDBDFB349B5F800000802C
:10BF600000100000000000000F610011997700111F
:10BF700033610011A17B0011B7610011777B0011C3
:10BF80002D6200114D7B00117F620011157D0011A3
:10BF9000E7620011157D001119630011CF7C0011BB
:10BFA0002D620011057B0011A5620011AD7C00110E
:10BFB00000000000000000008B630011AD7C001148
:10BFC000ED630011B1770011052A042A012A002A25
:10BFD0000229032801280028011800180000000089
:10BFE00000000000000000000000008701010201C5
:10BFF0000201010201020303040103010101010125
:10C000000303020103000D000E00100011001300D5
:10C010001401070108010A010B011C011D020402A1
:10C0200005020702080219021A021C021D0301037D
:10C03000020317000201000504000807000B0A00B4
:10C040001716001D1C010201010504010E0D01114E
:10C0500010011413011716011A19020201020B0A2A
:10C06000020E0D0211100214130217160305040329
:10C070000807030B0A030E0D0001020307090A0B50
:10C080000E0F101112141718191A1B1F202122004D
:10C09000F5A70011B1A80011000000000200000087
:10C0A000DABF001100000000DDB500110000000043
:08C0B00002000000D8BF0011DE
:020000041FFFDC
:1000000000000000ED3E001198BD001194BD0011EC
:100010003863FF1F00000000000000000000000027
:1000200000000000000000000000000000000000D0
:1000300000000000000000000000000000000000C0
:1000400000000000000000000000000000000000B0
:1000500000000000000000000000000000000000A0
:100060000000000000000000000000000000000090
:100070000000000000000000000000000000000080
:100080000000000000000000000000000000000070
:100090000000000000000000000000000000000060
:1000A0000000000000000000000000000000000050
:1000B0000000000000000000000000000000000040
:1000C0000000000000000000000000000000000030
:1000D0000000000000000000000000000000000020
:1000E0000000000000000000000000000000000010
:1000F0000000000000000000000000000000000000
:1001000000000000000000000000000000000000EF
:1001100000000000000000000000000000000000DF
:1001200000000000000000000000000000000000CF
:1001300000000000000000000000000000000000BF
:1001400000000000000000000000000000000000AF
:10015000000000000000000000000000000000009F
:10016000000000000000000000000000000000008F
:10017000000000000000000000000000000000007F
:10018000000000000000000000000000000000006F
:100190001535FF1F5D33FF1FC16601000000000021
:1001A000000000000000000000000000000000004F
:1001B000000000000000000000000000000000003F
:1001C000000000000000000000000000000000002F
:1001D000000000000000000000000000000000001F
:1001E000000000000000000000000000000000000F
:1001F00000000000000000000000000000000000FF
:1002000000000000000000000000000000000000EE
:1002100000000000000000000000000000000000DE
:1002200000000000000000000000000000000000CE
:1002300000000000000000000000000000000000BE
:1002400000000000000000000000000000000000AE
:10025000000000000000000000000000000000009E
:10026000000000000000000000000000000000008E
:10027000000000000000000000000000000000007E
:10028000000000000000000000000000000000006E
:10029000000000000000000000000000000000005E
:1002A000000000000000000000000000000000004E
:1002B000000000000000000000000000000000003E
:1002C000000000000000000000000000000000002E
:1002D000000000000000000000000000000000001E
:1002E000000000000000000000000000000000000E
:1002F00000000000000000000000000000000000FE
:1003000000000000000000000000000000000000ED
:1003100000000000000000000000000000000000DD
:1003200000000000000000000000000000000000CD
:1003300000000000000000000000000000000000BD
:1003400000000000000000000000000000000000AD
:10035000000000000000000000000000000000009D
:10036000000000000000000000000000000000008D
:1003700069B600110000000000000000000000004D
:10038000000000000000000000000000000000006D
:10039000000000000000000000000000000000005D
:1003A000000000000000000000000000951AFF1F80
:1003B000000000000000000000000000000000003D
:1003C000000000000000000000000000000000002D
:1003D000000000000000000000000000000000001D
:1003E000000000000000000000000000000000000D
:1003F00000000000000000000000000000000000FD
:081838006071FF1F4118FF1F42
:10184000024981F3088802F073FC00006071FF1FF9
:1018500010B502F05DFC072804D0122808D0022839
:1018600008D010BD044A0420136B01331363F8E75A
:101870000220F6E71420F4E73467FF1FF8B50700ED
:101880000C0026002500503630785135002804D150
:101890000300287058342370F8BD2978CA00481E08
:1018A0008141A3183800A25C5B68C9B2FFF7D0FF82
:1018B00000280DD12B78DA00A218013350602B706C
:1018C0003378044A013B3370136A01331362D8E75B
:1018D0000123DFE73467FF1F5C234343074910B54B
:1018E000C9180B0058331B78012B05D1FFF7C6FF31
:1018F000034A936A0133936210BDC0466867FF1FB5
:101900003467FF1F10B502F0D3FB064A0121130014
:1019100010CB4942D967044B136002F039FB200019
:1019200010BDC04600E100E01000100010B504003A
:1019300002F0BEFB024B1C6002F02AFB10BDC04649
:1019400000E100E010B5040002F0B2FB4021094ABA
:10195000200013688B43136002F0EAF901F0BCFD2C
:101960000022054B01201A60044B04321A6002F079
:101970004FFBFEE71CF00040C4F00040C0F0004008
:10198000431E5A425341A022F0B5D2015B4213409C
:10199000154D164A40019B182A18127E8BB00191F2
:1019A000002A1BD01A000832D46F0022E6B206AF1C
:1019B000E4B294420EDC2818C369002B08D00199C8
:1019C00002AA117106AA049202AA167303A89847E4
:1019D0000BB0F0BD1978B9540132EAE71A7D1A78D4
:1019E00006AB01261A70E6E7F469FF1F00400040CD
:1019F000F0B5254B04004001C25C85B0002A2BD015
:101A00001A18117E002927D0917E002924D011793F
:101A1000022921D11689D788D168F51BADB22A1CBD
:101A2000102D00D9102292B2BE4217D118180123EE
:101A300003710023C269C38003819A4206D06846BD
:101A4000032103730171029301A890470820002C21
:101A500000D0192001F038FC05B0F0BD013C654212
:101A60006C41A0256442ED012C40084D1B186419FF
:101A7000074D0633013A92B2AA42EDD01888461CAF
:101A80001E80085C2070F5E7F469FF1F00400040ED
:101A9000FFFF00000F220E4B10B59868104002386F
:101AA0000A280BD802F026F90D0A0B0A0A110A0AB5
:101AB0000A0A060002210020FFF762FF10BD012183
:101AC000F9E70020FFF794FFF8E7DB6FF6E7C04681
:101AD000004000400F220E4B10B5986810400238AD
:101AE0000A280BD802F006F90E0A0B0A0A120A0A93
:101AF0000A0A060002210120FFF742FF10BD012162
:101B00000800F9E70120FFF773FFF7E7DB6FF5E760
:101B10000090004013B5334C2378072B3DD8324B4F
:101B20001A78324B002A39D18022196852020A43AE
:101B30001A60252001F08CFF20232D4A11680B43E9
:101B4000802113606B460422C905086807331042E0
:101B500028D080210422C905C86810422ED08021D7
:101B60002020C905CA688243CA6014221A701A78F4
:101B7000002A2FD18021C905C86820320243CA60DB
:101B800014221A701A78002A28D11A4B1A7D22784A
:101B90005A601D221A705932DA6013BD1A6816494C
:101BA0000A40C5E7086802430A6014221A701A78CE
:101BB000002ACED01A78013AD2B2F7E7C8680243B9
:101BC000CA6014221A7019784A1ED2B21A700029FB
:101BD000F9D1C4E71A78013AD2B2C7E71A78013AC4
:101BE000D2B2CEE76445FF1F2C46FF1F3CF00040F9
:101BF0005C45FF1F00200040FFFFFEFF564B70B505
:101C00001B68012B03D1554A936D0133936502F094
:101C100097FA534B534A1860534B544C1A600123A4
:101C2000534A1360534A13602378002B06D00622D0
:101C30005149524802F0CCF900232370504A514BCD
:101C400010681B78C1B2002B0ED14F4CC0B2237864
:101C50005BB2002B4FDB237824785BB264B21B04A9
:101C600024021B191B1813600B1C50294ED950233A
:101C7000464A47491078DBB2FF2202284BD1086858
:101C8000444C454D267890432A78964254D9227880
:101C900024782E78023B5D10A31B6B435201D31AAC
:101CA00010335B111843086002F03AF9031F012B4F
:101CB00045D83A4B1B78002B06D0394B1B78002BAC
:101CC00002D0002002F03CF8A122364B9200997815
:101CD000354B4A431B689B18832292009B181B7844
:101CE000033B012B03D8AF20400002F061F9012231
:101CF0002E4BDA8270BD237824785BB264B2FF3356
:101D0000FF341B0424021B190138ABE7CAB2022AB4
:101D1000AED20223ACE70868254C264D26789043C6
:101D20002A78964208D9227824782D78023B5B10D5
:101D3000641B63435201B2E72378DBB2B2E70228A7
:101D4000D5D11D4B1B78013B022B03D91B4B1B78B4
:101D5000022BCCD16C20C8E79809FF1FFC0FFF1F96
:101D60006C66FF1FFF3F0000141003407066FF1FEA
:101D70000C10034000100340D50BFF1F7211FF1F12
:101D8000B40003408C09FF1F680AFF1F490AFF1FA8
:101D900094000340460AFF1F470AFF1FF908FF1F70
:101DA0002209FF1F300DFF1F3409FF1FBC0BFF1F4F
:101DB000440AFF1F450AFF1F1C09FF1F2309FF1FBD
:101DC00010B502F035F80022014B1A8010BDC04654
:101DD0006866FF1F10B502F0A3F9A121054A89002A
:101DE0009478054A61431268044B5218528C1A8049
:101DF00010BDC046300DFF1F3409FF1F6866FF1F6E
:101E000010B50D4B0D4A9978A1239B004B431268E6
:101E1000D218531DD97F0A4B1B88994209D2441C02
:101E200007D0C82805D0D2695B1A5A43054B5343E3
:101E3000C01802F00DFA10BD300DFF1F3409FF1F4E
:101E40006866FF1F7102000070B5244D2B68002BDF
:101E500028D002F0D5F82B68D8402B680400002B5E
:101E600027D002F08DF92B68D8401D4B1D4A997878
:101E7000A1239B004B431268D118D25C91239B0095
:101E8000002A20D0CA580132CA50174B17491B6884
:101E90000868834214D3D23B181A012A1AD0144B73
:101EA000186070BD02F0ACF8124B196802F0C0F86F
:101EB000D3E702F065F90F4B196802F0B9F8D4E7DF
:101EC0000D495B18E8E7CA500C4B1B68DB68E41847
:101ED000201AE4E7F530FF30E1E7C0461C08FF1F99
:101EE000300DFF1F3409FF1F9C09FF1F6C66FF1F89
:101EF000A009FF1F1808FF1F2DFF3F007466FF1F7A
:101F000070B504000D00282916D10300A433C2883F
:101F10001B889B1A0B4A9BB293420DD906006A3666
:101F200005223100653002F063F8002804D1310049
:101F3000200001F05DFF70BD2900200002F000F8D4
:101F4000F9E7C046FE7F0000F8B50400012002F06A
:101F50009FF801F0FDFF194A03001060184E194860
:101F6000016831600568A942FAD11748174E056823
:101F700077680020AF4201D27068281A144D091901
:101F800028601448C162A421446A49032143416284
:101F900011490978002905D010490978022902D190
:101FA0000F3B1360F8BD012901D1083BF9E7032974
:101FB00001D1053BF5E7033BF3E7C046E408FF1F0B
:101FC000340AFF1F28F00040180AFF1F28100040A5
:101FD0001C0AFF1F00F000401C09FF1F4A0AFF1FD8
:101FE00070B580241025E405A3682B43A36001F09D
:101FF000BFFFA368AB43A36070BD0000F7B5160038
:1020000080221C001023D2050191916805000B432A
:10201000936000225A4BD7301A6002F021F99D23B9
:102020002A002F009B00EB58CA3201210092FC3796
:10203000002B01D00021009A386801F051FF2900DF
:10204000009BCB311A784F4BD3351A604B780A7806
:102050001B0213438A7812041A43CB781B061343DE
:10206000494A1BBA13604B790A791B0213438A79D8
:1020700012041A43CB7931001B061343434A1BBA9F
:1020800013606B782A781B021343AA7812041A4350
:10209000EB781B0613433E4A1BBA1360019A3302C6
:1020A00013433C4A13603C4B22001B1B9C460329F4
:1020B0003DDCB3089A0013005142B21A032A46D1FC
:1020C000354AE018511A827840781204000202431F
:1020D000E05C043302430A600022FF2B4BDDF02258
:1020E0002E4B12011A600F222D4B1A602D4A1368D5
:1020F000002BFCD00023224A27491360091B321D04
:102100000B191B68043A180A23706070180C1B0E18
:10211000A070E3700434002AF2DC802210213B68B6
:10212000D20501333B6093688B439360F7BD6346F0
:10213000D578981893782D061B042B43157804390D
:102140002B43557804322D022B430360AFE7022A5C
:102150000AD1114AE05C511AE21852781202024385
:102160000A6004339BB2B7E7012AB5D10A4A521A72
:10217000E15C1160F5E7084959180A600433ACE7DF
:10218000000004403C000440380004403400044097
:10219000300004400C0004400001044004000440EE
:1021A0001000044014000440F7B5150080221C0004
:1021B0001023D2050091916807000B439360002320
:1021C000654AD730136002F04BF89D233E009B0018
:1021D000F9583B00CA363200FC33002900D07FE0BA
:1021E000586801F07DFE390032785C4BCB311A60C3
:1021F0004B780A781B0213438A78AC4612041A43C0
:10220000CB78281D1B061343554A1BBA13604B7924
:102210000A791B0213438A7912041A43CB791B06ED
:102220001343504A1BBA13604B7A0A7A1B021343BA
:102230008A7A12041A43CB7A21001B0613434A4AB6
:102240001BBA1360009A2B021343484A1360220002
:10225000474B1B1B0093009BCE785B1801938B7838
:1022600036061B0433430E78043833434E7804316A
:1022700036023343019E33600328ECDC0321A808B7
:10228000431C9B002940800003292BD13849E518C5
:102290005E18A9786D78E35C09042D02294319437F
:1022A0003160030008330021FF2B2DDD314B324913
:1022B00019600F21314B1960012327490B60304B06
:1022C00019680029FCD006211B680B40042B20D084
:1022D00080220020D20593680A318B439360FEBDB3
:1022E00001217DE7022908D121495D18E1184978CB
:1022F000E35C090219432960D3E70129D3D11C49C2
:102300005918E35C0B60CCE71948181801600433D6
:10231000CAE7002310490B606346002B0CDC3B002E
:10232000FC335A68102101325A608022D20593682A
:1023300001208B439360D2E7009B9B181B68190A0E
:1023400013705170190C1B0ED37004235B429170F3
:102350009C440432E0E7C046000004403C000440D6
:102360003800044034000440300004400C000440B5
:102370000001044004000440080F00001000044065
:102380001400044070B5061E19D00222614B9B79DF
:102390009343012B13D1604B1A78FF2A0FD15A783F
:1023A000FF2A0CD19A78FF2A09D1DA78FF2A06D1C0
:1023B0001A79FF2A03D15B79FF2B00D1A7E0574B95
:1023C0000C201A78012A08D00022554D1A702B785B
:1023D0001A00093A042A01D8212070BD5A1F012A87
:1023E000FAD94C4CA07B042800D990E0A279032AAA
:1023F00000D98CE0821E012A03D862881F2A00D8E7
:1024000085E0002E61D0012E00D080E0A288012A54
:10241000E2D0002B0AD10138032803D801F06AFC6E
:10242000151D19151F202E7001F0FAFC2B785A1E6D
:10243000032A16D800253B4B1D602823237501F085
:102440002FFEA8422ED0A580C6E7022320202B70A5
:10245000EAE7042322202B70E6E7032321202B70D8
:10246000E2E7073B012BB7D82F4B1B68DB6A9B06C3
:10247000B2D52E4B1A78002AAED1A27B911E01292B
:1024800001D9002AA8D1022280211A702823284DC0
:1024900089012878237501F02BFE80212878890195
:1024A00001F016FD0123A380224B1B78002B0AD0DC
:1024B000FA228021204B92001B8809025A431C4BB0
:1024C000187801F0FDFD002087E701F0F1FD2B7881
:1024D000A680073B012B06D918482E7001F090FC0E
:1024E0001E2001F09DFC114B114C1A78002A06D0D9
:1024F00080210022207889011A7001F0F9FD01F095
:1025000047FD80212078090201F0F2FDDBE712206F
:1025100063E7C046A60BFF1F6B09FF1F1A09FF1FC9
:102520001C09FF1F4809FF1F7466FF1F2309FF1FB7
:102530001B09FF1F2109FF1F2C09FF1F001000406E
:1025400010B5002901D001F0A3FC10BDF7B5604B18
:1025500001919978A1239B004B435E4A06001468C1
:102560001022E418D6235B00E0583623FF33E35CE7
:1025700000279343222B41D1574B0F3A1A60076033
:10258000012501F02DFD019B1880E8235B00E35C31
:10259000002B01D0B34258DD0023504FFB70AD3308
:1025A000FF33E3581A68002A03D09B88DB439B075C
:1025B0001DD03823FF33E35C002B18D09B235B0036
:1025C000E35C002B13D1D133FF33E35CB3420EDA6B
:1025D000A4235B00E15AE018090A023101F030FE41
:1025E00023000122FE33013E01351A87FA70E823E9
:1025F0005B00E35C002B2AD0A8B2FEBD03683D005F
:10260000002BBED081880430090A023101F018FE87
:10261000D6235B00E3581F60B2E72300B133BA0052
:10262000FF339858013781880430090A023101F0DC
:1026300007FEE8235B00E35CBB42EEDCE822F61A0F
:10264000ED1800235200A354A6E70027F1E720006D
:1026500001F006FD00281FD0002E1DDD731988260D
:1026600047190193B600200001F08AFB5A30800020
:1026700020184068013581880430090A023101F0D0
:10268000DFFD200001F06CFDA3590133A351BD42D1
:1026900002D0019B9D42E6D1114BE35C002BABD0F5
:1026A00095239B00E35C002BA6D00E4BE15A00293A
:1026B000A2D00D4AA35C994202D90133A3549BE7EF
:1026C00000231A212000A35401F062FB94E7C046C6
:1026D000300DFF1F3409FF1F00140340E010FF1FDF
:1026E0005A020000720200005E020000F8B51D4BA5
:1026F0001D4F1A78002A10D1BA7B002A02D101326C
:102700001A7003E0032AFAD0022AF8D001F0C8FCBC
:1027100000220120154B1A70F8BD154B154D1C6891
:10272000154B9E7801232B702878C0B200F0DEFC98
:10273000BB7B002B0BD101F0D3FCA1239B00734387
:10274000E41883239B00E41823782B70E4E7032B21
:1027500002D101F0ADFBF0E70020022BDCD101F04B
:1027600037FDEAE71C09FF1FA60BFF1F2309FF1F08
:102770003409FF1F490AFF1F300DFF1FF0B587B056
:102780000EAD2F780FAD2D780593AC46634614003F
:102790000E4D0CAA12782E7803930D9B0092019394
:1027A0002200059B029701F04BFC2E70012C01D0FA
:1027B000042C08D1802206498B889343054A12785D
:1027C000D20113438B8007B0F0BDC0461C09FF1F28
:1027D0006C11FF1F7809FF1F0B001B3B70B5040035
:1027E0003020E02B0DD81300E025493BFF3B9BB286
:1027F000ED00AB4205D8034B200019825A8201F04C
:10280000CFFA70BD8410FF1F10B501F099FC054B85
:1028100000205B68052B04D9034A5268D20200D419
:10282000980810BD00100040FCE100E070B501F018
:102830003FFC0D4B1B68FC33DC691D6AFFF7E4FFAE
:102840006419844204D2094B01241B68002B07D071
:1028500004220024064B1A70064A936901339361DF
:1028600001F096FB200070BD7466FF1F9809FF1FE2
:102870002309FF1FFC0FFF1F70B50C4D2B68FC33A5
:102880005C6A01F015FCFFF7BFFF2B680025FC33E5
:102890009B6AE318834204D2054B1B68AB4200D10C
:1028A000051B01F075FB280070BDC0467466FF1F54
:1028B0009809FF1FD722044B92009B5810B5002B9C
:1028C00000D0984710BDC0460000FF1FF0B587B08C
:1028D00001F09AF9FFF7EEFFCA4BCB4C04931B783B
:1028E000022B45D1C94B1B68186A01F0D1FBC84BBC
:1028F000C84A1A60C84BC94A1A60A022C84B520085
:102900001A60049B187801F0F3FAC649C64801F032
:10291000F7FAC649C64801F0F3FA1022C54BFF206A
:102920001A60802252031A60802292031A60802269
:1029300012041A6001F004FA012001F009FAFA20E9
:10294000400001F0E5FA582001F032FBBA4801F0EE
:1029500017FB012001F094FB072001F001FB226826
:10296000B64B1A4084235B001343236007B0F0BDCD
:1029700001F04EFAB24E0290322001F089FB33682A
:102980001B0629D43C2001F083FB0F2001F080FBC3
:102990009C4B1B78012B00D11EE180223368A94D8E
:1029A000134200D0A7E02B68032013432B6001F0F3
:1029B0006FFB01F02DFA029B0299C31A5A1E814245
:1029C00000D81A00A04B1A60904B19681E2353437D
:1029D0009E4A9B18CB618AE701F01AFA80239C4A31
:1029E000DB02116803900B4313602268934B994FED
:1029F0001A40282313432360032001F049FB0320DE
:102A00003D6801F045FB3B680320DB03DB0B0093D3
:102A100001F03EFB3B68ED03DB03ED0BDB0B8E4A65
:102A20000193AB18C22B30D8009B9B18C22B2CD81B
:102A3000019B9B18C22B28D8009B2A009D4200D2E4
:102A40001A00009B9D4200D91D00019B934200D2B9
:102A50001300019A954200D915005B1B122B14D864
:102A60000C22336814209343336033687B4A13404D
:102A7000336001F00DFB08213B682268DB038A43C9
:102A80002260774ADB0B13607FE7032001F000FB35
:102A90003B68DB03DB0B059301F0BAF9039B039959
:102AA000C21A531E814200D813006E4A93421BD9AA
:102AB000FF23356869492D0A1D4032686B1C1B06CF
:102AC0000A401B0C134333600C23326800209A43E6
:102AD000083B1343336001F0B3F96348634BA840EC
:102AE000984206DCFEF72EFF019B009D0093059B9C
:102AF00095E75F48F6E700235E4F554A3B60802329
:102B00001168DB020B43136080222B680320134300
:102B10002B6001F0BDFA3B68052601333B60802342
:102B20002A685B0213432B602268444B03201A403F
:102B3000514B1343236001F0ABFA0821454B1A684F
:102B40002368D2038B432360454B023900931B68F3
:102B5000D20B4B439A420CD89B1A3B2B0BD82368C1
:102B600046490B4023602B680B402B60444B1A6096
:102B70001FE7D31AF1E7013EF6B2002ED4D1236845
:102B80003E4A134023602B6813402B603B68042BA4
:102B900007D9BFF34F8F3B4B3B4ADA60BFF34F8FF0
:102BA000FEE780222B68032093432B6001F070FA2C
:102BB0002268224B03201A4028231343236001F08C
:102BC00067FA244B009A1B68DB03DB0B13600822B7
:102BD00023689343236097E707222C4D2B6813400B
:102BE000012B02D1002001F083F9AB68284A0220B2
:102BF0001340AB6001F04CFA8023AA685B001343DA
:102C0000AB60D6E64A0AFF1F5CF000407466FF1F07
:102C1000000003400180063DBC0003403408000072
:102C2000A40003407102000014100040FFFF3F00A9
:102C30002810004000E100E03075000000FEFEFFBB
:102C4000C4F0004044F000405C66FF1F72060000C4
:102C500040F0004064F0004091FCFFFFFF00FFFFE8
:102C60006466FF1FE30C0000E88000005F361E0072
:102C700060361E00C844FF1F28000100FFFFFEFF52
:102C80006066FF1F00ED00E00400FA053CF0004024
:102C9000FFFEFFFF694E336888331B6883F30888A3
:102CA00001F09EF800F018FC654B664A1B689342E1
:102CB00007D0002001F0C4F80221634A13688B4357
:102CC0001360FFF703FE614B614C1878C0B201F04E
:102CD000AFFA0023A3600233A3605E4B01202360A0
:102CE00001F0D6F90323A36001F092F8040001F08B
:102CF00027FA050001F08CF8574B186001F058F8DE
:102D0000564B1968621A531EA14200D2130080224A
:102D1000D203934201D39B029B0A3268D16AC9074E
:102D200000D478E04E491C0C09689BB24C435943CF
:102D30002402090A641803274A49FC3293680A6886
:102D400049489B1A494A4A4E12684A499B18414AC7
:102D500034609A183B400193036892089C46019B9B
:102D60000A6063440360042B03D901323B400A60CC
:102D700003600B684049E418200001F059F93F4F07
:102D80003D493B68C3183B602000019301F070F996
:102D90003B4C2068081838492060884205D9019BBF
:102DA00001333B6001F064F9216001F051F8354BCB
:102DB0001B78002B0ED001F0C3F93168324B4A1B4F
:102DC0001B6812189A4233D2591A4919091A2F4806
:102DD00001F096F82E4C237A002B0FD001F0B0F9B9
:102DE0003168E3684A1B1218934224D9591A4919C9
:102DF000091A284801F084F800232372264B83F334
:102E0000088801F0B5F9022001F00AF8002001F06D
:102E100017F801F0C5F9DC0199000234641A590071
:102E2000641A09214B438033CB40A408E41882E79D
:102E3000FA218900CBE71949DBE7C0467466FF1F1A
:102E40000C0AFF1FB641210310000040490AFF1F72
:102E500014100040C4090000100AFF1F340AFF1FAD
:102E6000380AFF1F200AFF1F280AFF1F1C0AFF1F26
:102E70005866FF1F240AFF1F710200006008FF1F31
:102E80002C0AFF1F1C09FF1FE408FF1F0010004051
:102E9000740BFF1F3C10004000000020DC05000008
:102EA000A022054B92009B5810B5002B01D09847EB
:102EB00010BD01F0B5F8FBE70000FF1FA122054B94
:102EC00092009B5810B5002B01D0984710BD01F01F
:102ED000A7F8FBE70000FF1FA222054B92009B58BA
:102EE00010B5002B01D0984710BD01F099F8FBE711
:102EF0000000FF1FA322054B92009B5810B5002B2A
:102F000001D0984710BD01F08BF8FBE70000FF1FD0
:102F1000A422054B92009B5810B5002B01D0984776
:102F200010BD01F07DF8FBE70000FF1F70B501F058
:102F300007F9514B1860042000F072FF01F068F9A6
:102F40000400C30702D401F033F970BD00224B4BDB
:102F50001A604B4B1878013804282CD800F0CAFEB0
:102F600003231B1F2700200000F08AFF0128ECD05C
:102F7000444C2378042B71D101F0C2F8002806D00C
:102F800000F09EFF582001F013F802232370032065
:102F900000F046FFD9E7200001F02AF9E6E720001B
:102FA00001F02EF9E2E7200001F03AF9DEE7200017
:102FB00001F006F9DAE700F0B3FF0500012808D1B7
:102FC000314B1B78053B012B03D82000FFF768FF2E
:102FD000CEE72C4B1B78022B01D0052B20D1022DE4
:102FE00028D12A4B9B7BAB431CD12000FFF766FF07
:102FF000254B18780128BBD16405B9D42349252273
:103000004B7B034205D1233A13405A4253412633A6
:103010001A000B7D9342ABD9322001F0E1F8A7E70B
:10302000022D07D1184B1B78052B11D12000FFF77B
:1030300053FFDDE7012D0BD1012B03D12000FFF75A
:1030400059FF95E7062B03D12000FFF761FF8FE7BB
:10305000200000F0E5FF022D8AD1C9E7032B04D13F
:103060000B4B987C00F004FF91E7072B8FD1094BA5
:10307000987B00F095FF8AE79C09FF1F9809FF1FC6
:103080009009FF1F2309FF1F1C09FF1FA60BFF1F2D
:10309000BC0BFF1FD40BFF1FFA210A4B0A4A490041
:1030A0001A640A4A5A500A4A04395A50094A0831DD
:1030B0009A64094A5A50094A5C315A50084ADA66F9
:1030C0007047C0460000FF1F7D27FF1F7928FF1FA4
:1030D0002D28FF1F8523FF1FED26FF1F011EFF1F49
:1030E000D51DFF1F10B500F0EDFD10BD8023F7B515
:1030F0009C46264B264F01932649274A274D284CAC
:10310000284B02281AD1604638600868264E3040A5
:10311000802636033043086001990978002909D1D7
:103120001660224A2A60224A2260E02219689143EE
:10313000A03A1BE08021C9021160F2E766463E60BA
:103140000F68194E3E408027FF023E430E600199F2
:10315000097800290DD1176001280ED1154A2A607F
:10316000154A2260E02219689143C03A0A431A6066
:10317000F7BD802189021160EEE7E0210F4A02438A
:103180002A600F4A22601A688A43F0E74B0AFF1F41
:10319000E0000340D80003409000034000000340DB
:1031A0005000034040000340FFFFE3FF0280063D64
:1031B000804508220180063D80660822008006982E
:1031C00080550822F8B51E4B80261A68002014008E
:1031D0003440324232D11A681A4F32431A60012207
:1031E0003B68063093433B6000F052FF0122164DCE
:1031F0002B681E432E603B680A2613433B608027E2
:10320000BF00124B1B683B4211D1013EF6B2FF2EAC
:1032100009D17E220E4B1C682B68E40B14409343AB
:1032200023432B6005E0082000F032FFE9E7002E81
:10323000EFD180222B68600893432B60F8BDC04615
:10324000C4F000405CF0004018F0004068F000401E
:1032500060F0004010B500F08BFD01215820034ABA
:1032600000F0F6FEFFF7AEFF10BDC046600AFF1F7C
:1032700010B578220021034800F0A2FE00F0F0FD16
:10328000002010BD7C69FF1F70B5040000F010FF26
:1032900000230C200B4A010059438D18515C002972
:1032A0000DD0A14208D1012300246B7000F010FF63
:1032B00000F06EFE200070BD01330A2BEBD112240A
:1032C000F6E7C0467C69FF1F70B5040000F0F0FE11
:1032D000002319001D000D4A1078002806D0A042D6
:1032E0000CD1557001310C320A29F5D1002B0AD1CD
:1032F00000F0B6FD00F04CFE002070BD5078461E78
:10330000B0411B18EEE700F0E3FEF3E77C69FF1F16
:10331000F7B504000C20002384460E4D0192674649
:103320005F43E85D7E19A04212D000280BD10A4B02
:103330009C4662461B7808331370019B70707C5565
:103340007160B360FEBD01330A2BE8D10320F9E7B9
:103350000720F7E77C69FF1F7869FF1F8020F8B519
:10336000484BC0051B68C1248360474BFF251A6882
:10337000012313434361454BA4001A68444B402189
:103380001A60444B1A68444B1A60444B1A59AA43BA
:103390001A51C52292009E58AE433143802699505F
:1033A0009F583F49F6010F403E439E509E5880274C
:1033B0003602360A3043985080201A5900020A40DB
:1033C00002431A5104341A59364E3F0432408026C3
:1033D0003A431A511A5936061202120A32431A5146
:1033E00008341A5980260A4002431A51C322920017
:1033F0009F58B446AF4337439F509F58294E0F40C4
:1034000007439F509F583740802636043743802615
:103410009F509F5836063F023F0A37439F50C022B5
:103420001F59AF433A431A511A591202120A16434E
:10343000C6221E5192009C58AC4365462C439C50BA
:103440009C5800250C4020439850C72080001A58F3
:10345000154C1140C02212020A431A50134B1B781C
:10346000DB08AB4201DC0020F8BD2378002B06D03E
:10347000A368002B00D0984701350C34EEE71220EA
:10348000F2E7C0466045FF1F5C45FF1FB0F00040FB
:103490007469FF1FB4F000407069FF1F00E100E095
:1034A000FF00FFFFFFFF00FF7C69FF1F7869FF1F20
:1034B000030010B51F2809D8072200201340072455
:1034C00004490A78A24313430B7010BD0023062061
:1034D000F5E7C0467869FF1F034A044913680020D6
:1034E0000B4013607047C0461CF00040FFFFC1FF57
:1034F000054B06491B780A6805485B0702401B0B11
:10350000134300200B6070477869FF1F1CF00040D8
:10351000FFFFC1FF70B50C25FFF7EAFF0A4B1C78CF
:103520000A4BE4086543ED18002C01D1200070BD62
:103530002B78002B06D06B68002B00D09847013CFD
:103540000C3DF1E71220F2E77869FF1F7069FF1F59
:1035500007B50422074801A900F034F9019B0133A3
:1035600005D18023044ADB0411680B43136000205B
:103570000EBDC0461C18001114F00040F0B5050047
:103580002026184B87B00493049B002B03D11124F1
:10359000200007B0F0BD002102220B000191009134
:1035A000052000F0D5FD02230F490A681A42FCD11C
:1035B0000596059C631E0593002CFAD10B4A1368EF
:1035C000002BFCDA0F276F440121380000F0A8FB24
:1035D0003B782B42DCD0052000F05AFD049B013BD8
:1035E0000493D1E7FFFFFF0790C8004000C80040E8
:1035F00007B500F05DFD80220821D205936A019194
:10360000002B01D10739916202210C4A1160019906
:10361000481E01900029FAD1033111600531019152
:103620000199481E01900029FAD11160002B02D1A6
:103630008022D205936200F0ABFC07BD00C00040C1
:10364000F0B52D4C89B02378002B4FD1FEF75AF9F5
:1036500002232A4F03903A681A42FCD12023069392
:10366000069B5A1E0692002BFAD1254E3368002B7A
:10367000FCDA0120FFF782FF011E02D0112009B001
:10368000F0BD030003220190009005AD9F2000F0E3
:103690005FFD0321280000F043FB02233A681A4231
:1036A000FCD120230793079B5A1E0792002BFAD1C7
:1036B0003368002BFCDA0120FFF760FF0028DDD122
:1036C0000398FEF733F9AA786B7811041B020B43B9
:1036D00029780B4363601300113B0A49052B07D877
:1036E00001239340A3600B60012323700020C6E7F1
:1036F00080231B03F6E7C0464845FF1F90C80040E3
:1037000000C800409808FF1F1E4B30B55A68187853
:103710001D4B85B0D31859424B4101210093002322
:1037200000F0BEFB194B1A4A02259A6300221A6563
:1037300010325A658022C4219D65164B1648D2026C
:10374000DA6789004258154B80241A4080231B04F5
:1037500013434350642341200393E40500F078F9B8
:10376000402000F075F96562039D6B1E0393002DE8
:10377000FAD103236362FFF73BFFA562FFF760FF07
:1037800005B030BD5445FF1F95FFFEF700C800404F
:10379000050001FF04E100E000E100E0FFFF00FFA1
:1037A00010B5064B18705960FFF7AEFF00211320CB
:1037B000034AFFF7ADFD002010BDC0465445FF1F72
:1037C0000937FF1FF0B5040085B003920291FEF7A0
:1037D00099F8882263035B0B52051A438023DB05AB
:1037E0009D6A8023274F0092BA68002601901B0330
:1037F0009A420CD9F82326001B041E401C4206D016
:103800008022214B52025E6219680A431A60002D21
:103810000BD100F04DFC02221C4B1A608023DB050B
:103820005A62013A9A6200F0B3FB0023039A934272
:1038300020D1002D0AD100F03BFC144B03221D6067
:103840008023DB055A629D6200F0A2FB8023BA68E8
:103850001B039A4208D9002E06D000220A4B0C49BD
:103860005A621A680A401A600198FEF75FF8002051
:1038700005B0F0BD009A0299D2181278CA540133EB
:10388000D4E7C0464845FF1F00C8004000C00040C4
:10389000FFFFFEFFF0B587B0029103920400FEF730
:1038A00031F8019000F004FC802302250122234E10
:1038B000DB0535605D629A6200F06AFB204F3B6871
:1038C0002B42FCD120230493049B5A1E0492002B0C
:1038D000FAD11C4D2B68002BFCDA0120FFF74EFEBD
:1038E000002802D0112007B0F0BD2000039A0299F1
:1038F00000F01EFB022304003A681A42FCD1202388
:103900000593059B5A1E0592002BFAD12B68002BBC
:10391000FCDA0120FFF732FE051EE3D100F0C8FB00
:1039200080230322DB0535605A629D6200F030FB84
:103930000198FDF7FBFFE0B2D5E7C04600C00040AC
:1039400090C8004000C80040F0B5802687B0040051
:10395000FDF7D8FFF605B36A02250393029000F045
:10396000A7FB0123244F3D607562B36200F010FB9A
:10397000224E33682B42FCD120230493049B5A1E11
:103980000492002BFAD11E4D2B68002BFCDA01208B
:10399000FFF7F4FD002802D0112007B0F0BD200091
:1039A00000F00EFA0223019032681A42FCD1202363
:1039B0000593059B5A1E0592002BFAD12B68002B0C
:1039C000FCDA0320FFF7DAFD041EE5D100F070FBFE
:1039D00080230322DB053C605A629C6200F0D8FA27
:1039E000039B002B01D1FFF703FE0298FDF79EFF1A
:1039F0006B461879D1E7C04600C0004090C800402F
:103A000000C8004007B5000201910422000A01A984
:103A1000FFF740FF0EBD000073B5050005240B4AFB
:103A2000A3005B429B1819686B46DE1D300000F056
:103A3000AFFB022804D133782B55013CEFD276BD81
:103A4000052CFCD00128FAD10230F8E71409001146
:103A50001F2807D8012380228340D20591680B4399
:103A6000936070473F2808D8012380222038834084
:103A7000D20551690B435361F3E75F28F1D8012365
:103A8000802240388340D205116A0B431362E8E775
:103A90001F2807D8012280218240C9058B689343E3
:103AA0008B6070473F2808D801228021203882404F
:103AB000C9054B6993434B61F3E75F28F1D80122B5
:103AC000802140388240C9050B6A93430B62E8E7C6
:103AD0001F2810D880230200DB05153A1968012A37
:103AE00006D820229143196019680A431A6070476A
:103AF00001228240F6E73F2811D880230200DB052F
:103B0000353AD968032A06D810229143D960D9687A
:103B10000A43DA60EBE7012220388240F5E75F28AC
:103B2000E5D842238022181A413B8340D205516ACE
:103B300099435162516A0B435362D8E710B50400B0
:103B4000012813D1A022184992050B685B015B097B
:103B500013430B60154B164A19681140154A0A4366
:103B60001A60402219680A431A6010BD0028FCD16F
:103B700001000A2000F02CF921000B2000F028F9A8
:103B8000C0220A4B920019680A4340211A601A6841
:103B90008A431A60B022044912060B685B015B0974
:103BA00013430B60E1E7C04614F000401CF00040F6
:103BB0007F00FEFF80FD010072B6074A13680133E3
:103BC00013600422054B1A600023054A136080220B
:103BD000D2055360FEE7C0467808FF1FC0F00040E2
:103BE000C4F00040044B054A1A60054B1A600022DD
:103BF000044B1A607047C046140AFF1F841E000061
:103C0000380AFF1FC4F000400023034A1360034A30
:103C10001360034A1360704754F0004040F10040C5
:103C200044F10040002310B5184C8AB00093019372
:103C30002378012B27D06946012000F091F8002855
:103C400017D1009B12490293019B06AA0393114BC3
:103C500002A81B680493104B1B68059300F088F9B9
:103C600010220E4906A800F0C3F9002804D1FF2352
:103C7000237000200AB010BD0123094A074902A899
:103C8000237000F075F90120F4E7C0467866FF1F45
:103C900010290011082900110C29001120290011F8
:103CA0007C66FF1F13B501246946012000F058F817
:103CB000034B00940193FFF7B5FF200016BDC046EB
:103CC000BB0B000010B5FFF79FFFFFF7EBFF0028CD
:103CD00002D0024B984710BDFEE7C046E1A20000AB
:103CE00002B4714649084900095649008E4402BC95
:103CF0007047C04602B4714649084900095C490052
:103D00008E4402BC7047C04603B471464908400067
:103D10004900095A49008E4403BC70470000000066
:103D200001B40248844601BC604700BF3D710100F8
:103D300001B40248844601BC604700BFF9A60000F8
:103D400001B40248844601BC604700BFED6B01002E
:103D500001B40248844601BC604700BF69110100FC
:103D600001B40248844601BC604700BFE1AC0000DA
:103D700001B40248844601BC604700BFED68010001
:103D800001B40248844601BC604700BFD9B00000BE
:103D900001B40248844601BC604700BF53B900002B
:103DA00001B40248844601BC604700BF116E0000A8
:103DB00001B40248844601BC604700BFC1660100EF
:103DC00001B40248844601BC604700BFA96F0100EE
:103DD00001B40248844601BC604700BF89A20011BB
:103DE00001B40248844601BC604700BFC9A9000075
:103DF00001B40248844601BC604700BF85C1000091
:103E000001B40248844601BC604700BFC1A5000060
:103E100001B40248844601BC604700BF156B010035
:103E200001B40248844601BC604700BF1907010085
:103E300001B40248844601BC604700BF8D82000087
:103E400001B40248844601BC604700BF016C010018
:103E500001B40248844601BC604700BFD54401005C
:103E600001B40248844601BC604700BFADAE00000B
:103E700001B40248844601BC604700BF4DF9000010
:103E800001B40248844601BC604700BF0134010010
:103E900001B40248844601BC604700BFE9D4000079
:103EA00001B40248844601BC604700BFC56D0100F3
:103EB00001B40248844601BC604700BF75F80000A9
:103EC00001B40248844601BC604700BF6DF60000A3
:103ED00001B40248844601BC604700BF0D52010096
:103EE00001B40248844601BC604700BF2144000081
:103EF00001B40248844601BC604700BFEDA5000044
:103F000001B40248844601BC604700BF2D6C01002B
:103F100001B40248844601BC604700BF851201001D
:103F200001B40248844601BC604700BFDD0C0100BB
:103F300001B40248844601BC604700BF957301008C
:103F400001B40248844601BC604700BF51B800007C
:103F500001B40248844601BC604700BFBD5C01005B
:103F600001B40248844601BC604700BFF90D01005E
:103F700001B40248844601BC604700BFDD3F000039
:103F800001B40248844601BC604700BF8D110100A6
:103F900001B40248844601BC604700BF9DA90000EF
:103FA00001B40248844601BC604700BFC1F700006D
:103FB00001B40248844601BC604700BF7912010089
:103FC00001B40248844601BC604700BFB70E000040
:103FD00001B40248844601BC604700BFE94C0100BF
:103FE00001B40248844601BC604700BFCD0C01000B
:103FF00001B40248844601BC604700BFCD4C0100BB
:1040000001B40248844601BC604700BFE90B0100CF
:1040100001B40248844601BC604700BFA1AF000064
:1040200001B40248844601BC604700BFE9170100A3
:1040300001B40248844601BC604700BF090E00007D
:1040400001B40248844601BC604700BF9D6A00007D
:1040500001B40248844601BC604700BF016701000B
:1040600001B40248844601BC604700BF71B0000043
:1040700001B40248844601BC604700BF090E00003D
:1040800001B40248844601BC604700BFE51201004C
:1040900001B40248844601BC604700BF01890000AA
:1040A00001B40248844601BC604700BFA9D80000A3
:1040B00001B40248844601BC604700BF75A90000F6
:1040C00001B40248844601BC604700BF8B52010026
:1040D00001B40248844601BC604700BF21A900002A
:1040E00001B40248844601BC604700BFE9F6000005
:1040F00001B40248844601BC604700BFB3520100CE
:1041000001B40248844601BC604700BF01D70000EB
:1041100001B40248844601BC604700BFE9270000A3
:1041200001B40248844601BC604700BFF9ED0000BD
:1041300001B40248844601BC604700BF75B6001157
:1041400001B40248844601BC604700BFC95C01005D
:1041500001B40248844601BC604700BF496D0100BC
:1041600001B40248844601BC604700BF5976010093
:1041700001B40248844601BC604700BF7997000043
:1041800001B40248844601BC604700BF6D0B0100CA
:1041900001B40248844601BC604700BF8D3800115D
:1041A00001B40248844601BC604700BF855201004B
:1041B00001B40248844601BC604700BFDD0A01002B
:1041C00001B40248844601BC604700BFF9350100D4
:1041D00001B40248844601BC604700BF19FA0000E0
:1041E00001B40248844601BC604700BF613701004A
:1041F00001B40248844601BC604700BF0934010095
:1042000001B40248844601BC604700BF0534010088
:1042100001B40248844601BC604700BFBD0B0100E9
:1042200001B40248844601BC604700BFF535010077
:1042300001B40248844601BC604700BF89140100F4
:1042400001B40248844601BC604700BFC1150100AB
:1042500001B40248844601BC604700BF89370100B1
:1042600001B40248844601BC604700BF8944000095
:1042700002000000D6BF00110100000088BD00113F
:1042800002000000D2BF001101000000B042FF1F79
:104290000200000090BD001101000000B863FF1F84
:1042A00002000000D0BF0011030000002C63FF1FBC
:1042B0001200000002000000D6BF00110100000043
:1042C000D0BD001102000000D2BF001101000000AB
:1042D000CDBD001102000000DABD00110300000096
:1042E0006763FF1F02000000D0BF00110300000041
:1042F0007C63FF1F02000000D2BF0011010000001C
:10430000CCBD001102000000D8BD00110300000068
:104310003D63FF1F02000000D0BF0011030000003A
:104320005E63FF1F02000000D6BF00110100000005
:1043300010BE001102000000D2BF001101000000F9
:10434000F943FF1F0200000022BE0011010000001F
:104350000BBE001102000000D2BF001101000000DE
:10436000F843FF1F0200000020BE00110100000002
:104370008463FF1F02000000D2BF00110100000093
:10438000F743FF1F020000001EBE001101000000E5
:10439000FBBD001102000000D2BF001101000000AF
:1043A000F643FF1F020000001CBE001101000000C8
:1043B000F6BD001102000000D2BF00110100000094
:1043C000F543FF1F020000001ABE001101000000AB
:1043D000F1BD001102000000D2BF00110100000079
:1043E000F443FF1F0200000018BE0011010000008E
:1043F000ECBD00110202020202020000414C001159
:10440000074C001164BE0011900118001800FFFF56
:104410000701020304050602010600000000000077
:10442000000000000000000000000000000000008C
:10443000000000000000030002000000D6BF0011D1
:1044400001000000E4BE001102000000D2BF001114
:1044500001000000A844FF1F02000000EEBE001192
:1044600001000000B263FF1F02000000D0BF001176
:10447000030000002066FF1F02000000D2BF0011F1
:1044800001000000A844FF1F02000000ECBE001164
:1044900001000000B463FF1F02000000D0BF001144
:1044A000030000001866FF1F12A6A6A60000000069
:1044B0000001000000000111FFFF000050485936C4
:1044C00000000000000000000100000075BE0011A7
:1044D0000B000500F7000000B400002800280028A9
:1044E0003075A000A000A000A00000080008E001B6
:1044F000F00010001000100010001000100050001C
:104500005000500010001000D00700000000000014
:104510000F0001000500307507001000010081FF49
:1045200000000000FF00000071740011797200119A
:1045300009700011FFFF0100FF0000008D9E0011B7
:10454000099C0011219B00110000000000000000E8
:1045500000000800040000003B0001085902E001CF
:1045600088212800FF00000002000000D6BF0011D3
:10457000010000009CC0001102000000D2BF001129
:1045800001000000E545FF1F02000000CEBF001142
:1045900001000000346AFF1F02000000D2BF0011BA
:1045A00001000000E445FF1F02000000CCBF001125
:1045B00001000000E245FF1F02000000D2BF001111
:1045C00001000000E045FF1F02000000CABF00110B
:1045D00001000000D845FF1F1800180000009001DE
:1045E000020000030202000002000000D6BF00111A
:1045F00001000000B0C0001102000000D2BF001195
:10460000010000002846FF1F02000000C8BF001183
:10461000000000000000000002000000D0BF0011F8
:0A46200003000000546AFF1F20FF92
:040000051FFF184180
:00000001FF
